:020000040800F2
:10000000183B0020B1010008CB3A0008652B00081E
:10001000C93A0008890300081562000800000000C2
:10002000000000000000000000000000253E000865
:100030006104000800000000473C0008ED3E000895
:10004000CB010008CB010008CB010008CB01000860
:10005000CB010008CB010008CB010008CB01000850
:10006000CB010008CB010008CB010008CB01000840
:10007000CB010008CB010008CB010008CB01000830
:10008000CB010008CB010008CB01000800000000F4
:10009000000000000000000000000000CB0100088C
:1000A000CB010008CB010008CB010008CB01000800
:1000B000CB010008CB010008CB010008CB010008F0
:1000C000CB010008CB010008CB010008CB010008E0
:1000D000CB010008CB010008CB01000800000000A4
:1000E000CB010008CB010008CB0100080000000094
:1000F000000000000000000000000000CB0100082C
:1001000000000000CB010008CB010008CB01000873
:1001100000000000000000000000000000000000DF
:10012000CB010008CB010008CB010008CB0100087F
:10013000CB010008000000000000000000000000EB
:10014000000000000000000000000000CD3A0008A0
:10015000CB010008CB010008CB010008CB0100084F
:10016000CB010008CB0100080000000000000000E7
:10017000000000000000000000000000000000007F
:1001800000000000CB01000800000000000000009B
:10019000CB010008CB010008DFF810D000F0A4F874
:1001A0000048004791640008AFF30080183B00202E
:1001B0000648804706480047FEE7FEE7FEE7FEE701
:1001C000FEE7FEE7FEE7FEE7FEE7FEE7813F000809
:1001D000990100082DE9F05F0546002092469B46F4
:1001E00088460646814640241BE02846414647464D
:1001F000224600F068F853465A46C01A914110D37F
:1002000011461846224600F04FF82D1A67EB0108F8
:100210004F4622460120002100F046F817EB000966
:100220004E41201EA4F10104DFDC484631462A4637
:100230004346BDE8F09F40EA01039B0703D009E075
:1002400008C9121F08C0042AFAD203E011F8013BC2
:1002500000F8013B521EF9D27047D2B201E000F81B
:10026000012B491EFBD270470022F6E710B513465A
:100270000A4604461946FFF7F0FF204610BD421C0F
:1002800010F8011B0029FBD1801A704710B500221D
:1002900000E0521C835C8C5CA34201D1002BF8D19E
:1002A000D8B2E1B2401A10BD202A04DB203A00FA8D
:1002B00002F1002070479140C2F1200320FA03F3BD
:1002C000194390407047202A04DB203A21FA02F0BB
:1002D0000021704721FA02F3D040C2F12002914080
:1002E0000843194670470000064C074D06E0E068D9
:1002F00040F0010394E8070098471034AC42F6D36D
:10030000FFF74EFF2CA100084CA100080EB50A23F0
:100310000092CDE9011302460123A021014800F01B
:1003200011FE0EBD200100200EB50A230092CDE97A
:10033000011302460123A021014800F005FF0EBD74
:100340002001002008B500250BA005F0C7FD8DF8A1
:1003500000500024684605F08FFD28B19DF800008C
:10036000302801D103F0E8F90A2000F011FB641CE9
:10037000322CEFDBE8E7000023235049434F5F4274
:100380004F4F5423230D0A00FEE700207047002042
:100390007047000010B500220449054804F0DAF85F
:1003A0000449034804F0C9F8002010BD101C0020C7
:1003B000340700201014002070B500220B4C0C4BA9
:1003C00008E0855C1E88A5551D886D1CC5F30A05CF
:1003D0001D80521C0D689542F3D80146054804F073
:1003E000ACF8044804F082F8002070BD100C002026
:1003F000760000203407002000207047094A10B51D
:10040000D2F8BC22D2F814220AB1012010BD0A464B
:100410000146044804F09EF8BDE81040014804F08D
:1004200013B90000340700203EB50B4A04460D46C0
:10043000106840F480501060106800F48050029002
:1004400006480090684600F05AFAAA082146684615
:1004500000F03EFA3EBD000030380240003002405D
:10046000704708B50A2000F093FA6A46022100207E
:10047000FFF74CFF9DF80000552803D19DF80100BF
:10048000AA2821D055208DF80000AA208DF801005F
:100490000A2000F07DFA6A4602210020FFF744FF9F
:1004A000002000900A2000F073FA6A460221002022
:1004B000FFF72CFF9DF80000552803D19DF801009F
:1004C000AA2801D0012008BD002008BD0EB50020DB
:1004D0000090019002906A4608212020FFF716FF45
:1004E00004A16846FFF7D2FE08B100200EBD01202E
:1004F0000EBD00007570646174650D0A0000000097
:100500000EB510B107A007C801E009A207CA8DE81F
:1005100007006846FFF7B3FE81B26A462020FFF766
:1005200003FF0EBD7570646174650D0A0000000064
:100530002D6E6F70652D0D0A0000000072B6FEE78B
:10054000002229B101291AD002291BD04FF4407290
:100550000E490B6823F440730B600B6813430B6068
:100560000A6822F0F8020A600A68022303EBC0005E
:1005700002430A60086840F48030086070474FF416
:100580008072E5E74FF40072E2E70000103C0240A1
:100590001348016889050FD5016821F400710160D5
:1005A000016841F400610160016821F400610160AB
:1005B000016841F400710160016849050FD50168C7
:1005C00021F480610160016841F48051016001689B
:1005D00021F480510160016841F48061016070473D
:1005E000003C024038B50220009001240A4800F087
:1005F00031F9C0088440C4F58050009000F032FA10
:100600000121009800F092F800F020FA08B10220D1
:1006100038BD012038BD00000000010810B586B0CB
:100620000B4800F017F90446002000900294094896
:1006300000F010F9001B401C03900220049005A953
:10064000684600F0B7F9002800D0012006B010BDC0
:1006500000000108FFFF070800B587B000210290E5
:100660000120039002200091049005A9684600F043
:10067000A1F9002800D0012007B000BD10B508483E
:1006800000F0E8F807490988C008C14040F6FF7249
:10069000C240914201D1012010BD002010BD0000D8
:1006A00000000108163C024010B500F0DBF90249D9
:1006B000F320086010BD00000C3C02402DE9F04121
:1006C00016468846054600240D4F11E058F82410C0
:1006D000286800F03BF82868016858F82400814237
:1006E00002D00220BDE8F0812868001D2860641C4B
:1006F000B44202D22868B842E8D90020F2E70000EC
:10070000FBFF070808490A6822F440720A600A6879
:1007100042F004020A600A684FF4803343EA002082
:1007200002430A6070470000103C024010B50446C6
:100730004CF2503000F05AF8002803D102490A88E0
:1007400022430A8010BD0000163C0240074A13688D
:1007500023F440731360136843F400731360136849
:1007600043F001031360016070470000103C024039
:100770001C490868C2061C4805D5C26942F010022F
:10078000C26110220A600A68920605D5C26942F069
:100790000802C26120220A600A68520605D5C269B1
:1007A00042F00402C26140220A600A68120605D5BE
:1007B000C26942F00202C26180220A600A68D20560
:1007C00006D5C26942F00102C2614FF480720A602C
:1007D0000A68920705D5C26942F02002C261022070
:1007E000086070470C3C02401402002070B51149AB
:1007F00004460020C86100F0DBFA06460E4D09E011
:10080000601C07D024B100F0D3FA801BA04201D9AC
:10081000032070BD2868C003F2D42868C00701D047
:1008200001202860286810F4F970F2D0FFF7A0FFCB
:10083000012070BD140200200C3C024008B50020CD
:100840008DF80000684605F017FB0028FAD09DF8E7
:10085000000008BD01460020A1F100634FF4804272
:10086000934204D314480844904201D201207047B7
:1008700012480844904201D20220704710480844B0
:10088000904201D2032070470E480844B0F5803FE3
:1008900001D2042070470C480A184FF400308242FD
:1008A00001D205207047094A1144814201D2062035
:1008B000704707207047000000C0FFF70080FFF777
:1008C0000040FFF70000FFF70000FEF70000FCF714
:1008D00030B50223437103689C6844F001049C60B6
:1008E000002304E0056851F823402C605B1C934210
:1008F000F8D30168096801224271084630BD10B57D
:10090000040002D0607910B106E0012010BD002083
:100910002071204600F004F801206071002010BD15
:1009200008B500680649884208D10648016841F4C4
:1009300080510160006800F48050009008BD000004
:1009400000300240303802400E4910B50C480860B3
:1009500000200860091D0C4A0A60086009490B4A1A
:1009600010390A6008608022091D0A600860421E72
:10097000091D0A60086000F0F5FC002010BD0000B1
:100980000FC8E21020380240317917009F10600034
:1009900070B5044600F00CFA0546601C02D004480D
:1009A0000078044400F004FA401BA042FAD370BD62
:1009B000080000202DE9F047044622480F46017E3A
:1009C00001290AD00121804601764CF2503948466F
:1009D000FFF70CFF020003D02FE00220BDE8F087F4
:1009E0004FF0FF3038602068174D012801D0A6680D
:1009F0001CE0207C6168FFF785FE4846FFF7F6FEA5
:100A00000246286820F00400286014E0217C30466B
:100A1000FFF796FD4846FFF7E9FE0200286820F040
:100A2000FA00286001D03E6005E0761CD4E902108F
:100A30000844B042EAD8FFF7ABFD002188F818104F
:100A40001046CBE714020020103C02400448017815
:100A500041F0020101704CF25030FFF7C7BE0000B8
:100A6000143C0240074900200A68002A09DA054AB6
:100A7000054B0C3A1360054B13600968002900DA36
:100A800001207047103C024023016745AB89EFCD40
:100A90002DE9F04F0022DFF808B101264FF00F09D1
:100AA00006FA02F401EA0403A34274D122F0030718
:100AB0005F44D7F8088895074FEA157C09FA0CFAC5
:100AC0000AEA0805DFF8DC80404502D14FF0000853
:100AD0001DE0DFF8D480404502D14FF0010816E058
:100AE000DFF8C880404502D14FF002080FE0DFF880
:100AF000C080404502D14FF0030808E0DFF8B48021
:100B0000404502D14FF0040801E04FF0070808FA11
:100B10000CF8A84522D1284DD5F800C02CEA030CCA
:100B2000C5F800C02D1DD5F800C02CEA030CC5F88F
:100B300000C0214D0C35D5F800C02CEA030CC5F8D7
:100B400000C02D1FD5F800C02CEA030CC5F800C06A
:100B5000D7F8085825EA0A05C7F808580568570065
:100B60000323BB409D430560D50800EB8505D5F800
:100B700020C057074FEAD76809FA08F72CEA070C94
:100B8000C5F820C0C5689D43C5604568A54345605C
:100B900084689C438460521C102A81D3BDE8F08F86
:100BA0000030014000000240000402400008024002
:100BB000000C024000100240003C01402DE9F84FBB
:100BC000DFF8B8A10022012403254FF00F090AF134
:100BD000040BAAF1040E00BF0B6804FA02F63340BE
:100BE000B34273D10F7907F00307012F01D0022F11
:100BF00016D187684FEA420805FA08FC27EA0C0775
:100C0000D1F80CC00CFA08FC4CEA070CC0F808C07C
:100C10004768B7430E79C6F3001696403E434660D8
:100C20000E79F643B6070DD0C768560005FA06FCE4
:100C300027EA0C07D1F808C00CFA06FC4CEA070CAE
:100C4000C0F80CC00E7906F00306022E10D1D608AB
:100C500000EB8608D8F8206057074FEAD76C09FAEE
:100C60000CF7BE430F6907FA0CF73743C8F820703A
:100C700006684FEA420C05FA0CF7BE430F7907F0FD
:100C8000030707FA0CF7374307604E6816F4403F36
:100C90006DD03B4E376847F480473760366822F0A6
:100CA000030706F480460096364E07EB060CDCF888
:100CB000086897073F0F09FA07F826EA0806DFF8E1
:100CC000C880404503D14FF000081EE04FE0DFF838
:100CD000BC80404502D14FF0010816E0DFF8B0803B
:100CE000404502D14FF002080FE0DFF8A8804045F0
:100CF00002D14FF0030808E0DFF89C80404502D1A4
:100D00004FF0040801E04FF0070808FA07F848EA36
:100D10000608CCF80888DAF800605746D1F804C015
:100D20009E435FEACC2C00D51E433E60DBF800609A
:100D30005F46D1F804C09E435FEA8C2C00D51E4369
:100D40003E60DEF800607746D1F804C09E435FEA5B
:100D50008C3C00D51E433E60084F083F3E68D1F8EA
:100D600004C09E435FEACC3C00D51E433E60521C4B
:100D7000102AFFF431AFBDE8F88F0000083C0140B5
:100D800044380240003001400000024000040240AC
:100D900000080240000C02400010024000690840B8
:100DA00000D0012070470AB1816170470904FBE758
:100DB00001488068704700000800002070B50400FA
:100DC00025D094F83D00002520B984F83C502046F9
:100DD00000F052FA242084F83D002068016821F0D8
:100DE000010101602068016841F400410160206850
:100DF000016821F40041016001F0C2F94D4A6168C7
:100E0000914201D84C4900E04C49884201D201206E
:100E100070BD4B492368B0FBF1F15E6826F03F06D8
:100E20000E435E606368934206D94FF4967359434C
:100E30004FF47A73B1FBF3F12368491C1E6A26F064
:100E40003F06314319626168914210D84900401E43
:100E5000B0FBF1F2521CC2F30B02042A01D20420AF
:100E600022E0B0FBF1F0401CC0F30B001CE0A268D4
:100E7000F2B301EBC10303EB0116431EB3FBF6F320
:100E80005B1C43F480431B0549D092B301EBC102C4
:100E900002EB0111401EB0FBF1F0401CC0F30B004F
:100EA00040F4804040F400402168CA694CF6FF736A
:100EB0009A431043C861D4E90710014320680268CF
:100EC00022F0C00211430160D4E90301014320680C
:100ED000826848F2FF339A4311438160D4E90501E7
:100EE00008432168CA6822F0FF021043C86001E08D
:100EF0000EE016E02068016841F001010160256400
:100F0000202084F83D00256384F83E50002070BD09
:100F100001EB4106431EB3FBF6F35B1CB3E7012074
:100F2000C2E701EB4101401EB0FBF1F0401CC0F3F1
:100F30000B00B7E7A086010080841E0000093D0079
:100F400040420F002DE9FF4F83B09A46DDE911873B
:100F500093460446DDF84090FFF72AFF054694F8D3
:100F60003D00202870D119230122744920460095A4
:100F700001F00EFF0028F5D194F83C00012863D061
:100F8000012084F83C0020680168C90703D101688A
:100F900041F0010101602068016821F400610160F5
:100FA000222084F83D00402084F83E00002626647C
:100FB000C4F82490A4F82A80608D20856048E062FF
:100FC000CDE9007553465A462046049901F0E2FDEA
:100FD000002879D1208DD0B1012821D002282068A5
:100FE00024D0416980690090208D032866D80128AB
:100FF0002BD0544902283B464FF00002009557D0B1
:101000008846204601F0C4FE00285DD13AE0206801
:10101000416981690091016841F4007101607DE0DE
:101020002068016821F480610160F0E7016821F423
:10103000806101602068016841F4006101602068FE
:1010400041698069009069E075E02A46394620468A
:1010500001F044FF88BB54E02068016841F400714E
:10106000016020680069616A0870606A401C606203
:10107000218D491E2185618D491E6185216809697F
:10108000017042E02068016821F4806101602068FD
:101090000069616A0870606A401C6062208D401EB1
:1010A0002085608D401E60853B46002241460095AC
:1010B000204601F06DFE00B9CEE705E02A4639462C
:1010C000204601F00BFF18B1012007B0BDE8F08FFA
:1010D00020680069616A0870606A401C6062208D47
:1010E000401E81B22185608D401E60852068426966
:1010F000D243520712D4032903D1016821F480613D
:10110000016020680069616A0870606A401C606262
:10111000208D401E2085608D401E6085208D00281A
:101120007FF462AF202084F83D0084F83E6084F8AC
:101130003C600020C9E70220C7E700000200100061
:101140000000FFFF040001002DE9FF4F83B09A4625
:10115000DDE9119793460446DDF84080FFF728FE4D
:10116000054694F83D0020287FD1192301224049EB
:101170002046009501F00CFE002876D194F83C0042
:10118000012872D0012084F83C0020680168C9075A
:1011900003D1016841F0010101602068016821F478
:1011A00000610160212084F83D00402084F83E0069
:1011B00000262664C4F82480A4F82A90608D208537
:1011C0002C48E062CDE9007553465A462046049902
:1011D00001F05EFD70B930E02A463946204601F044
:1011E000B5FE58B1206C042804D12068016841F490
:1011F00000710160012007B0BDE8F08F606A2168CE
:1012000000780861606A401C6062218D491E89B2C5
:101210002185628D521E628522685369DB435B071C
:101220000BD469B100781061606A401C6062208D47
:10123000401E2085608D401E6085208D0028CBD10A
:101240002A463946204601F077FD0028CAD154F8D5
:101250003D0B016841F400710160202004F81E0973
:10126000E67766770020C6E7FFE70220C3E70000C5
:10127000020010000000FFFF10B586B004461421E4
:101280006846FEF7F1FF13492068884220D11248D2
:101290000021026842F002020260006800F00200D1
:1012A0000590C02000901220CDE901010320039099
:1012B0000420049069460948FFF780FC0648103076
:1012C000016841F400110160006800F4001005900D
:1012D00006B010BD00540040303802400004024007
:1012E000024881680278114481607047080000203C
:1012F0000B4810B5016841F400710160016841F4C8
:1013000080610160016841F480710160032000F098
:1013100081F80F2000F006F800F026F8002010BD3C
:10132000003C024070B50D4D04464FF47A712878A8
:10133000B1FBF0F00A490968B1FBF0F001F06BFA7B
:1013400048B9102C07D200222146501E00F042F866
:1013500000206C6070BD012070BD000008000020FE
:1013600014000020704700000A4808B5016841F4E5
:1013700080410160006800F4804000900548001F33
:10138000016841F080510160006800F080500090D9
:1013900008BD00004438024000280DDB00F01F02A9
:1013A000012191404009800000F1E020C0F8801147
:1013B000BFF34F8FBFF36F8F7047002809DB00F03A
:1013C0001F02012191404009800000F1E020C0F897
:1013D00000117047F0B40E4B1B680C46C3F3022398
:1013E000C3F10705042D00D90425191D072901D2D1
:1013F000002300E0DB1E012606FA05F1491E21400C
:1014000099409E40761E16403143F0BC04F0C2BFA6
:101410000CED00E0064900F0070208684FF6FF03F4
:10142000184040EA0220034A104308607047000059
:101430000CED00E00000FA057047006841620020F2
:101440007047F0B50368586A39B19C6A4FF48276E8
:1014500000EB144400204D1E0AE040EA024098626E
:101460000FE006EB8007DF59401C04EB1744C0B2C5
:10147000A842F6D344EA02404FF4807202EB8101A5
:1014800058500020F0BDD0F8E00403F093BB01EB0E
:10149000C10200EB8202D0F8E004126A03F0DFBA66
:1014A00001EBC10200EB8202D0F8E004D2F8602226
:1014B00003F030BB10B5040006D0032084F8950477
:1014C000206804F023FE08B1012010BD204600F082
:1014D0002DFC002084F8950410BDD0F8E00403F042
:1014E0006BBB0A0601F00F0101EBC10100EB8101AA
:1014F00001D5143101E001F51571006804F01CBC40
:1015000070B504460B0601F00F0000EBC00104EBC0
:1015100081014FF001024FF0000502D54A751431E8
:1015200003E081F8555201F51571087094F89404A0
:10153000012808D084F89424206803F05BFF84F825
:101540009454002070BD022070BD70B5044601F0B7
:101550000F002279904201D9012070BD0B0601F0E5
:101560000F0101EBC10104EB81014FF001024FF0CB
:10157000000502D54A75143103E081F8555201F592
:1015800015718D70087094F89404012808D084F8BF
:101590009424206804F05CFA84F89454002070BD10
:1015A000022070BD01F00F0101EBC10100EB8100D1
:1015B000D0F8680270472DE9F04104460F0601F0AB
:1015C0000F0000EBC00104EB81014FF001064FF06A
:1015D000000502D54E75143103E081F8555201F52E
:1015E0001571C2F30A0208708A600B714A7802B161
:1015F0004883022B00D14D7194F89404012809D03E
:1016000084F89464206803F047FE284684F89454D4
:10161000BDE8F0810220FBE710B501F00F0404EBF8
:10162000C40100EB8101C1E998230023C1F86832AD
:1016300081F8553281F85442837901F51571012BF7
:1016400000D1CA618279006804F05AFA002010BD06
:1016500070B504460D4601F00F002179884201D98A
:10166000012070BD29064FF000064FF0010206D59B
:1016700000EBC00104EB81014A75143107E005EB72
:10168000C50104EB810181F8556201F515718A707D
:10169000087094F89404012807D084F894242068F2
:1016A00004F002FA280702D007E0022070BDA179F9
:1016B00004F29C42206804F09FF984F894640020AE
:1016C00070BD10B501F00F0404EBC40100EB810103
:1016D000C1E9082300238B6201234B7501F8144FE5
:1016E0008379012B00D1CA618279006804F008FA7D
:1016F000002010BD2DE9FC5F05680446284604F073
:10170000B7FB00287DD1206804F02AFC002878D09F
:10171000D5F80808C0F30D20C4F8D404206804F0FC
:101720001FFC800704D52068416901F00201416176
:10173000206804F015FCC10604F29C40009034D5EA
:101740002068816921F0100181612F6A07F00F0084
:1017500000EBC00004EB8006C7F3434006F51576A6
:10176000022802D0062811D01AE047F6F07007428E
:1017700016D0C7F30A1217462846F16804F0F4FBA6
:10178000F0683844F0607069384408E00822284660
:10179000009904F0E9FB7069C7F30A11084470610D
:1017A0002068816941F010018161206804F0D8FB54
:1017B00000034FF0080B4FF0000A4FF001097CD5F1
:1017C0000026206804F0ABFB074674E0F80770D0F1
:1017D000F1B2206804F0BCFB8046C00707D005EBDF
:1017E0004611C1F8089B3146204602F075F95FEAC0
:1017F000087024D505EB4611C1F808BB2068016CC0
:1018000000E023E200EB46100191D0F8082BFB4BDF
:10181000994205D9110403D54FF40041C0F8081BC3
:10182000204600F00DFBF5490198884207D9A079C0
:10183000012804D120680121009A04F0DDF85FEA54
:10184000C86004D505EB46111020C1F8080B5FEA0B
:1018500088701DD56869000605D5D5F8040840F4E0
:101860008061C5F8041806EBC60004EB800090F810
:10187000571200F51570012905D180F803A0F1B2C7
:10188000204600F0E9F905EB46110220C1F8080BEB
:101890005FEA886004D505EB46102021C0F8081BDC
:1018A0005FEA884005D505EB46104FF40051C0F8BB
:1018B000081B7F08761C002F88D1206804F050FB9D
:1018C00040036ED5206804F023FB0746002666E03F
:1018D000F80762D0F1B2206804F028FB8046C00708
:1018E00023D006F00F01D5F8342809FA01F18A4314
:1018F000C5F8342805EB4611C1F80899A0790128EC
:101900000FD106EBC60004EB8000D0E9072111449B
:10191000016236B9606A20B920680121009A04F09A
:101920006BF8F1B22046FFF7B2FD5FEA087003D50D
:1019300005EB4611C1F808B95FEAC86004D505EBAC
:1019400046111020C1F808095FEA486004D505EB8C
:1019500046104021C0F808195FEA887016D5314654
:10196000284604F05AFA06EBC60004EB8000C17D5D
:101970001430012905D180F803A0F1B2204600F00F
:1019800067F905EB46110220C1F808095FEA086013
:1019900003D53146204602F005F97F08761C002F5A
:1019A00096D1206804F0DCFA002811DAD5F8040892
:1019B00020F00101C5F8041894F8CC0401282BD0BC
:1019C000204600F022FA2068416901F0004141619F
:1019D000206804F0C5FA00050BD5D5F80808C00743
:1019E00002D0204600F07AFA2068416901F40061D3
:1019F0004161206804F0B4FAC00467D5D5F8040842
:101A000020F00100C5F804081021206804F005FA50
:101A100000214FF67F3220E084F8CCA4002120463C
:101A2000FFF70AFDCFE700BF05EB4110C0F808291A
:101A3000D0F8003923F40013C0F80039C0F8082B9F
:101A4000D0F8003B23F40013C0F8003BD0F8003B73
:101A500043F00063C0F8003B491C20798842E3D87A
:101A6000D5F81C0840F00111C5F81C18E07B0028CF
:101A700028460DD0D0F8840840F00B01C5F8841832
:101A8000D5F8440840F00B012846C5F844180DE08D
:101A9000D0F8140842F22B010843C5F81408D5F811
:101AA000100840F00B012846C5F81018D0F80008BF
:101AB00020F4FE61C5F80018A1792068009A03F0AF
:101AC0009BFF2068416901F480514161206804F066
:101AD00047FA800415D5206803F01EFC206804F046
:101AE000BAF9E07100F046FB0146E279206804F0A3
:101AF00099FA204600F076F92068416901F4005116
:101B00004161206804F02CFA000707D5204600F058
:101B100080F92068416901F008014161206804F002
:101B20001FFA000616D5A86920F08001A9610126D8
:101B30000DE000BF06EBC60004EB800090F85702F2
:101B4000012803D1F1B22046FFF7CBFC761C2079A7
:101B5000B042EFD8206804F003FAC0021FD5012676
:101B60004F4614E005EB4610D0F8001906EBC6000E
:101B700004EB8002107E012808D1002906DAF0B2B9
:101B800040F08001D7752046FFF7ABFC761C20792A
:101B9000B042E7D82068416901F4801141612068B2
:101BA00004F0DEF9800234D501204A4629E000BF66
:101BB00005EB4011D1F8001B00EBC00304EB8303DD
:101BC00093F85862012E1BD1002919DA94F8D464D5
:101BD00001F4803106F00106B14211D183F8572299
:101BE000A96941F08003AB616969090608D4D5F899
:101BF000040840F40070C5F8040805E00A30544FAA
:101C0000401C21798142D3D82068416901F4001138
:101C10004161206804F0A4F9400007D52046FFF791
:101C200032FC2068416901F080414161206804F084
:101C300097F940070AD520684568680702D520460D
:101C4000FFF74BFC2068416829434160BDE8FC9FD9
:101C5000D0F8E00403F003B8D0F8E00403F013B8C0
:101C6000F8B5040005D094F895042668002510B155
:101C700006E00120F8BD84F89454204600F070F886
:101C8000032084F89504B6F1A04F00D1A571206817
:101C900003F0F0FC207C8DF8000094E80F0003F0C6
:101CA00049FB0226B8BB0021206804F07CF990BBF8
:101CB000002001270DE000BF00EBC00104EB810113
:101CC0004F750875C8850D76CD610D62401CC0B298
:101CD0004D6221798142EFD8002011E000EBC00174
:101CE00004EB810181F8555281F8540281F8585271
:101CF000C1F85C52C1F86052401CC0B2C1F86452D5
:101D000021798142EAD8207C8DF8000094E80F0008
:101D100003F0F2FB10B184F89564AAE7657484F8C7
:101D20009574206803F0DAFB0020F8BD10B5006858
:101D3000B0F1A04F0ED10848016821F08001016088
:101D40004FF4C0510548FEF7A3FEBDE81040432004
:101D5000FFF722BB10BD00003438024000000240F3
:101D600010B586B0044614216846FEF77DFA206857
:101D7000B0F1A04F2FD119480021026842F00102B2
:101D80000260006800F0010005904FF4C050009020
:101D90000220CDE90101032003900A200490694646
:101DA0000F48FEF70BFF0D48001D016841F0800150
:101DB00001600A481430016841F480410160006804
:101DC000002200F48040059011464320FFF702FBFB
:101DD0004320FFF7F2FA06B010BD00003038024091
:101DE0000000024070B50446C0790125022801D0E8
:101DF000FEF7A4FB2946D4F8E00402F0B2FFD4F8C1
:101E0000E004BDE8704002F067BFD0F8E00402F0E3
:101E100091BFD0F8E00402F097BF10B5044690F8E7
:101E2000940401280AD0012084F894046174206885
:101E300004F0E7F8002084F8940410BD022010BDDF
:101E4000D0F8E02400F29C41104602F096BF10B595
:101E50000446006894F89414012909D0012184F8FB
:101E60009414C168490609D5617B012902D005E0B7
:101E7000022010BD816B41F480318163206803F042
:101E8000AAFF206803F01CFB002084F8940410BD16
:101E900070B50446006894F894140546012912D0E0
:101EA000012184F8941403F0E5FB206803F016FB8D
:101EB0001021206803F0B1FFE868400609D5607B77
:101EC000012802D005E0022070BDA86B20F480300C
:101ED000A863002084F8940470BD000010B5044687
:101EE000D0F8E00402F094FF2068D0F8001E41F022
:101EF0000101C0F8001EE07A002804D00248016801
:101F000041F00601016010BD10ED00E02DE9F04741
:101F10000E46050065D0DFF81481D8F80000F7B24E
:101F200000F00700B04207D288F80070D8F800002F
:101F300000F00700B04254D128683D4C810712D50B
:101F4000400703D5206840F4E0502060287800075F
:101F500003D5206840F4604020602068A96820F024
:101F6000F000084320602878C0072DD03049686809
:101F70000839012812D0022813D0032811D009688B
:101F8000890700292DDA216821F00301014321602E
:101F9000FEF70EFF814641F2883A0EE00968890398
:101FA000EFE709688901ECE7FEF702FFA0EB090102
:101FB000514502D90320BDE8F0872068696800F028
:101FC0000C00B0EB810FEFD1D8F80010404601F0C3
:101FD0000701B14207D90770006800F00700B0425E
:101FE00001D00120E7E72878400705D52068E96897
:101FF00020F4E050084320602878000706D52068C8
:10200000296920F4604040EAC100206000F0C8F86F
:102010002168084AC1F30311515CC84006490860B1
:1020200006480068FFF77EF90020C4E7003C024044
:1020300008380240989F0008140000200C0000207F
:102040002DE9F041FEF7B4FE444C0546206840F00F
:102050000100206005E000BFFEF7AAFE401B022839
:1020600047D820688007F7D5206840F080002060BE
:10207000FEF79EFE0546394E00200836306041F2DC
:10208000883704E0FEF794FE401BB84231D8306830
:1020900010F00C0FF6D1FEF78BFE0546206820F4F9
:1020A0005020206005E000BFFEF782FE401B642840
:1020B0001FD820688003F7D4FEF77AFE0546206813
:1020C00020F08070206004E0FEF772FE401B0228C2
:1020D0000FD820688001F7D4FEF76AFE0546206815
:1020E00020F08060206007E0FEF762FE401B0228BF
:1020F00002D90320BDE8F08120680001F4D417491B
:102100001748091D086015491648843108601348AE
:102110000C30016821F4F8510160016821F400518C
:102120000160016841F41F010160016841F4001180
:1021300001600A487430016821F001010160016802
:1021400041F080710160094907480860084800684B
:10215000FFF7E8F80028CDD00120CBE70038024097
:1021600010300004103000200024F400140000207F
:102170000C00002001480068704700001400002097
:102180000448054900680968044AC1F38221515C8A
:10219000C84070471400002008380240A89F00087B
:1021A000154810B5006810F00C02144813D01449FB
:1021B000042A0FD0082A0ED10F4C241F226823684E
:1021C00002F03F025B0207D52068C0F38810A0FB35
:1021D000010106E0084610BD2168C1F38811A1FB8A
:1021E00000010023FDF7F6FF2168C1F30141491CFE
:1021F0004900B0FBF1F010BD083802400024F400A3
:1022000040787D012DE9F84F04006ED02078DFF88A
:102210004C93C007A9F104054AD009F104000168F4
:10222000C1F38101012908D00068C0F381000228B0
:102230000AD1D9F80000400206D52868800337D5B6
:1022400060680028E1D033E06068B0F5803F10D0CE
:10225000B0F5A02F286810D020F4803028602868BE
:1022600020F4802028606068A8B1FEF7A1FD064632
:102270000DE0286840F48030F4E740F480202860C6
:10228000F7E700BFFEF794FD801B642873D8286829
:102290008003F7D50CE0FEF78BFD064605E000BF96
:1022A000FEF786FD801B6428F0D828688003F7D4E9
:1022B0002078DFF8AC8280074FF0000A3ED5A748AF
:1022C000001D016811F00C0F08D00068C0F38100F8
:1022D00002280BD1D9F80000400207D428688007F3
:1022E00016D5E068012800D112E033E1E068B8B10A
:1022F0000120C8F80000FEF75BFD064605E000BFC0
:10230000FEF756FD801B0228C0D828688007F7D545
:102310002868216920F0F80040EAC10028600DE03B
:10232000C8F800A0FEF744FD064604E0FEF740FDB5
:10233000801B02281FD828688007F7D42078000760
:1023400022D5864F87486169703771B101210160DC
:10235000FEF72EFD064604E0FEF72AFD801B02284C
:1023600009D838688007F7D50EE0C0F800A0FEF75E
:102370001FFD064605E082E0FEF71AFD801B0228DD
:102380007DD838688007F7D42078400768D5DFF813
:10239000CCB100270BF13C0BDBF80000C0000BD4E4
:1023A000DBF8001041F08051CBF80010DBF80000A2
:1023B000012700F0805000906B4E3068C00510D4AB
:1023C000306840F480703060FEF7F2FC009005E069
:1023D000FEF7EEFC0099401A022850D83068C0057C
:1023E000F6D55E4EA0686C3601280FD005283068FF
:1023F00010D020F001003060306820F00400306020
:10240000A068B8B1FEF7D4FC00900FE0306840F04F
:102410000100F4E740F004003060F7E7FEF7C8FC85
:102420000099411A41F28830814266D830688007AD
:10243000F4D50EE0FEF7BCFC009007E0FEF7B8FC18
:102440000099411A41F28830814256D8306880079D
:10245000F4D42FB1DBF8001021F08051CBF800103C
:10246000A069C8B33D49091D0968C1F3810102296A
:102470004AD00228504607D0C8F8600000E03CE08F
:10248000FEF796FC04463BE04746C8F86000FEF7BE
:102490008FFC064605E000BFFEF78AFC801B022881
:1024A0002BD828688001F7D4D4E907010843A16A32
:1024B0002E4A490802EB0141626A41EA821108434F
:1024C00094F82C1040EA0161C9F800100120386628
:1024D000FEF76EFC044606E03EE000BFFEF768FC37
:1024E000001B022809D828688001F7D534E000BF16
:1024F000FEF75EFC001B022802D90320BDE8F88F1E
:1025000028688001F4D427E00128F7D0D9F800002A
:10251000E26900F4800191421CD1226A00F03F017F
:10252000914217D147F6C071626A0140B1EB821F38
:1025300010D1A26A4FF0FF3300F4403103EB520296
:10254000B1EB024F06D194F82C1000F07060B0EBA4
:10255000016F01D00120D1E70020CFE7043802400D
:1025600000004742800E4742007000400000FFFF1D
:1025700070B5040009D0606A002540B1256165612D
:10258000A56294F8510040B10CE0012070BD606874
:10259000B0F5827FF4D0E561F2E784F85050204630
:1025A00000F044F8022084F851002068016821F00E
:1025B00040010160A088218900F4827001F4044187
:1025C0000843A18901F400610843217C01F0020164
:1025D0000843217D01F001010843218B01F40071C2
:1025E0000843217F01F03801084394F8201001F0DE
:1025F00080010843218D01F40051084321680860DF
:10260000A069042101EA104094F8241001F010019F
:102610000843216848602068C16921F40061C161F4
:102620006565012084F85100002070BD10B586B0AA
:10263000044614216846FDF717FE144920688842B5
:1026400021D113480021026842F4804202600068F0
:1026500000F4804005900E481038026842F00202F3
:102660000260006800F0020005904FF420400090E6
:102670000220CDE901010320039005200490694662
:102680000448FEF79BFA06B010BD00000038004079
:1026900040380240000402402DE9F84F98461646A3
:1026A0008A460446FEF784FB814694F851000128CF
:1026B0001ED1BAF1000F73D0002E71D094F85000E3
:1026C000012815D0012784F85070032084F85100A8
:1026D00000256565C4F830A0A686E686A563A587B3
:1026E000E58765642564A068B0F5004F03D00CE071
:1026F0000220BDE8F88F2068016821F040010160E8
:102700002068016841F48041016020680168490641
:1027100003D4016841F040010160E068B0F5006F4A
:10272000606803D048B3012E27D047E008B1012EDE
:102730001FD1206B21680088C86006E0206881688E
:10274000890709D5216B0988C160206B801C206333
:10275000E08E401EE0860CE0FEF72AFBA0EB0901AC
:10276000414503D3B8F1FF3F03D035E0B8F1000F86
:1027700032D0E08E0028E1D123E0206B2168007880
:10278000087306E02068816889070AD5216B0978FB
:102790000173206B401C2063E08E401EE0860DE03C
:1027A0002BE0FEF705FBA0EB0901414503D3B8F18F
:1027B000FF3F03D010E0B8F1000F0DD0E08E0028ED
:1027C000E0D14A464146204601F09AFA08B120205D
:1027D0006065A06830B109E084F8517084F8505009
:1027E000032086E72068C1688068009084F85170F3
:1027F00004F8505F60680028F3D0012079E74FF0BB
:10280000E0210428086903D020F004000861704723
:1028100040F00400FAE710B5401EB0F1807F01D30C
:10282000012010BD4FF0E02460610F21601703F01C
:10283000B1FD0020A06107202061002010BD10B56F
:1028400090F83C20012A22D0012280F83C20CA685E
:102850008C6822F4407222434C6822F48062224346
:102860000C6822F4006222430C6922F48052224355
:102870004C6922F400522243C969002322F48042A9
:102880000A4301684A6480F83C30002010BD0220F1
:1028900010BD000070B590F83C20012A2CD0012416
:1028A00080F83C40022280F83D2003685A689D6809
:1028B00022F070060A6832435A60104B02689A424E
:1028C0000ED0B2F1804F0BD00D4B9A4208D00D4B79
:1028D0009A4205D00C4B9A4202D00C4B9A4204D13A
:1028E000496825F080031943916080F83D4000213C
:1028F00080F83C10084670BD022070BD0000014009
:102900000004004000080040000C0040004001406E
:1029100010B586B0044614216846FDF7A5FC0E49A3
:102920002068884216D10D480021026842F0010259
:102930000260006800F0010005904FF48060009094
:102940000220CDE901010120CDE9031069460448C8
:10295000FEF734F906B010BD0000014030380240E7
:102960000000024070B5044690F83C0000260D4679
:1029700001280FD0012084F83C006AB1042A1DD040
:10298000082A2FD00C2A3FD00126002084F83C00D2
:10299000304670BD022070BD206801F059FB2068F0
:1029A000816941F0080181612068816921F0040199
:1029B0008161206881692A69114311E0206801F072
:1029C0006FFB2068816941F4006181612068816941
:1029D00021F480618161206881692A6941EA0221CC
:1029E0008161D2E7206801F087FB2068C16941F06E
:1029F0000801C1612068C16921F00401C16120683A
:102A0000C1692A69114311E0206801F0A1FB206827
:102A1000C16941F40061C1612068C16921F480612C
:102A2000C1612068C1692A6941EA0221C161ACE73C
:102A300010B5040003D094F83D0010B107E0012068
:102A400010BD002084F83C00204600F01FF8022052
:102A500084F83D00211D206801F09AFA012084F8D5
:102A6000460084F83E0084F83F0084F8400084F873
:102A7000410084F8420084F8430084F8440084F85C
:102A8000450084F83D00002010BD000008B5006836
:102A90000649884208D10648016841F001010160F9
:102AA000006800F00100009008BD00000000014037
:102AB0004438024010B50446022249B104290ED020
:102AC000082913D094F84100012816D0012010BD28
:102AD00094F83E000128F9D184F83E200FE094F8E4
:102AE0003F000128F2D184F83F2008E094F840002C
:102AF0000128EBD184F8402001E084F84120012234
:102B0000206801F097FA12492068884203D1426C8C
:102B100042F400424264206888420ED0B0F1804FF7
:102B20000BD00C49884208D00B49884205D00B498C
:102B3000884202D00A49884204D1816801F0070125
:102B4000062903D0016841F001010160002010BD99
:102B5000000001400004004000080040000C00405C
:102B600000400140FEE701684A69D24352050FD494
:102B70006FF480624A61002140F8301F20224273C6
:102B80008173026942F004020261017301207047FF
:102B9000002070472DE9F84F0446006889460B9DD8
:102BA00001689846174641F4806101602068016819
:102BB00041F48071016000954FF0011B00225946DD
:102BC00020460A9B00F0E4F84FF4007A40B12068F8
:102BD0000068C00501D5C4F840A00320BDE8F88F07
:102BE000216809F0FE0008612B46284920460A9A10
:102BF00000F016F9F0BB20684169806900902A4610
:102C000020460A9900F0A2F940B1206C04283AD17C
:102C10002068016841F40071016034E0FEB2B8F14F
:102C2000010F09D02168380A08612A4620460A990E
:102C300000F08CF90028E8D1206806612A46204679
:102C40000A9900F083F90028DFD12068016841F477
:102C50008071016000950022594620460A9B00F0D1
:102C600097F80028B3D1216809F0FF0040F0010077
:102C7000086100E007E02B46044920460A9A00F06C
:102C8000CFF80028AAD00120A8E700000200010028
:102C90002DE9F843044600680D46DDE90897016810
:102CA0009846164641F4807101604B4600224FF071
:102CB00001112046009700F06BF848B120680068C9
:102CC000C00502D54FF4007020640320BDE8F883EE
:102CD000216805F0FE0008613B464A46154920463A
:102CE00000F09EF888B920684169806900903A46F2
:102CF0004946204600F02AF948B1206C042804D146
:102D00002068016841F4007101600120DEE7F5B23E
:102D1000B8F1010F09D02168300A08613A464946E6
:102D2000204600F013F90028E7D120680561002053
:102D3000CCE700000200010070B516460D460446BF
:102D40001EE02046FFF70FFF08B1012070BD681C90
:102D500016D0FEF72DF8801BA84200D885B9206850
:102D60004069C04340070BD5002044F8300F2021B4
:102D70006173A073216941F0200121612073E4E7B0
:102D800020684069C0434007DBD4002070BD0000CC
:102D90002DE9F047984617460D460446C1F307460D
:102DA000DDF820902AE000BFB8F1FF3F26D0FDF704
:102DB000FFFFA0EB0901414502D8B8F1000F1DD17A
:102DC0002068012E16D0806925EA00000004000C5E
:102DD00012D00020B84211D1002044F8300F202139
:102DE0006173A073216941F02001216120730120EA
:102DF000BDE8F0874069E7E70120EBE72068012E96
:102E00000AD0806925EA00000004000C06D00020EA
:102E1000B842C9D00020EBE74069F3E70120F7E7AB
:102E20002DE9F047984616460D4604464FF0000936
:102E30004FF0200AC1F3074723E020684069C043F0
:102E4000400515D42068016841F4007101602168D3
:102E50006FF480604861C4F8309084F83DA084F835
:102E60003E90216C41F00401216484F83C9021E003
:102E7000701C06D0FDF79CFFA0EB0800B04203D801
:102E800016B1012F1FD021E02068012F15D08069D5
:102E900025EA00000004000C18D000BF44F8309F61
:102EA00084F80DA084F80E90216941F02001216181
:102EB00084F80C900120BDE8F087406925EA000005
:102EC0000004000CEAD12068406901E020688069B4
:102ED00025EA00000004000CAFD1ECE72DE9F04139
:102EE000002590460E460446202728E04069C0434E
:102EF000C0060CD454F8301B6FF01000486144F841
:102F000010596777A577206A2062257714E0FDF7CE
:102F10004FFFA0EB0800B04200D886B92068406996
:102F2000C04340060BD544F8305F6773A573206932
:102F300040F02000206125730120BDE8F081206869
:102F40004169C9434906D1D40020F6E770B5164659
:102F50000D4604461EE02046FFF705FE08B101209D
:102F600070BD681C16D0FDF723FF801BA84200D857
:102F700085B920684069C04300060BD5002044F89D
:102F8000300F20216173A073216941F0200121617C
:102F90002073E4E720684069C0430006DBD40020CA
:102FA00070BD0000F0B500220D4B154614460A27EF
:102FB000B1FBF3F630368654B1FBF3F603FB161182
:102FC000B3FBF7F3521C861816F8016C302E00D1B3
:102FD00025B16D1C641C0A2CEAD3F0BD0022F9E770
:102FE00000CA9A3BF0B500230A24302537261F4635
:102FF00011E000BFB4EB107F02D905EB107C01E0BB
:1030000006EB107C01F813C001EB430C00015B1CC4
:103010008CF80170DBB29342ECD3F0BD00B587B001
:1030200014216846FDF720F909480021026842F0A2
:1030300001020260006800F0010005900120CDE966
:103040000001029069460348FDF7B8FD07B000BDD6
:1030500030380240000002402DE9F04104461D4690
:1030600016460F462A2000F023FA204600F010FAF8
:10307000304600F00DFA2B2000F01AFA384600F026
:1030800007FA284600F004FABDE8F0412C2000F0D1
:103090000FBA10B5503114468BB289B20246FFF711
:1030A000DBFF2046BDE8104000F0F2B92DE9F04703
:1030B00080461F4603F14F0083B21646501E82B26F
:1030C0000C4601F1500081B24046DDF82090FFF738
:1030D000C3FF0AE0454604E0484600F0D9F96D1CFC
:1030E000ADB2B542F8D3641CA4B2BC42F2D3BDE881
:1030F000F0870000F0B587B014216846FDF7B4F8FA
:103100001848016841F002010160016801F0020104
:103110000591016841F00201016000684FF480569A
:1031200000F00200059001240F4FCDE90064032553
:10313000694603953846FDF741FD01223146384680
:10314000FDF731FE2E02CDE90064084C6946039577
:103150002046FDF733FD012231462046FDF723FED0
:1031600007B0F0BD303802400004024000000240C9
:1031700070B5FFF7BFFF00224FF480716748FDF77D
:1031800012FE674D4FF48054002221462846FDF779
:103190000AFE642003F034F9012221462846FDF797
:1031A00002FE642003F02CF9112000F081F9782050
:1031B00003F026F9362000F07BF9C02000F08EF9EC
:1031C0003A2000F075F9052000F088F9B22000F0EF
:1031D0006FF90C2000F082F90C2000F07FF900203C
:1031E00000F07CF9332000F079F9332000F076F913
:1031F000B72000F05DF9352000F070F9BB2000F039
:1032000057F9192000F06AF9C02000F051F92C207C
:1032100000F064F9C22000F04BF9012000F05EF9E3
:10322000C32000F045F9122000F058F9C42000F046
:103230003FF9202000F052F9C62000F039F90F20A4
:1032400000F04CF9D02000F033F9A42000F046F94A
:10325000A12000F043F9E02000F02AF9D02000F08E
:103260003DF9042000F03AF90D2000F037F9112063
:1032700000F034F9132000F031F92B2000F02EF982
:103280003F2000F02BF9542000F028F94C2000F0EA
:1032900025F9182000F022F90D2000F01FF90B206D
:1032A00000F01CF91F2000F019F9232000F016F996
:1032B000E12000F0FDF8D02000F010F9042000F02B
:1032C0000DF90C2000F00AF9112000F007F9132085
:1032D00000F004F92C2000F001F93F2000F0FEF886
:1032E000442000F0FBF8512000F0F8F82F2000F007
:1032F000F5F81F2000F0F2F81F2000F0EFF8202072
:1033000000F0ECF8232000F0E9F8212000F0D0F8DC
:10331000BDE87040292000F0CBB80000000002405A
:1033200000040240411F5F2909D84FF4967110FB39
:1033300001F06421B0FBF1F001490968C8637047EE
:10334000CC0100202DE9FF4F81B00446DDF83C9010
:1033500000904FEA59074FF00008780700D001208D
:1033600000EBD70000FB09FB203AD0B20390029893
:1033700048444F3083B2E019401E82B20298503068
:1033800081B22046FFF768FE002553E0B9F10C0F2B
:103390002AD0B9F1100F2ED0B9F1180F2ED0B9F1F3
:1033A000200F49D12749039801EB8010002610F81F
:1033B00005A0109800284FF0010000FA06F000EA7E
:1033C0000A0022D020B12046049A0299FFF761FE3C
:1033D000641C0098A4B2201AB84225D10298009C1F
:1033E000401C80B2029023E00398174900EB400094
:1033F00001EB8000DAE71549039803E003981449CC
:1034000000EB400001EB0010D0E708B1049800E0A9
:103410000E9800F03DF808F10100C0B2B0FBF7F1E2
:10342000804607FB118050B1761CF6B2082EC0D33F
:103430006D1CADB25D45A9D305B0BDE8F08F4FF06E
:103440000008F5E7B08200087C660008F06A000812
:10345000E07000082DE9FE4F9946DDE90D6714463E
:103460008A460546DDF830800CE0CDF800804B46FA
:1034700051462846CDE90167FFF764FF05EB56008A
:1034800085B2641C2278002AEFD1BDE8FE8F0000CF
:1034900008B5010A8DF800108DF801000123022201
:1034A00069460248FFF7F8F808BD000074010020E3
:1034B00070B5094D06464FF4007400222146284697
:1034C000FDF771FC304600F009F821462846BDE8BA
:1034D00070400122FDF767BC0000024001B50123E6
:1034E0001A4669460148FFF7D7F808BD7401002065
:1034F000074910B5054808600846FDF700FA00289E
:1035000003D0BDE81040FDF719B810BD00300240EF
:10351000000000202DE9F04186B014216846FCF738
:10352000A3FE23480024016841F004010160016802
:1035300001F004010591016841F08001016001681A
:1035400001F080010591016841F00201016001680C
:1035500001F002010591016841F00101016000687C
:10356000012200F00100134F55030590294638460B
:10357000FDF719FCDFF84080EE100022314640468E
:10358000FDF711FC00950125CDE901546946384647
:103590000394FDF713FB0220CDE90204CDE9006599
:1035A00069464046FDF70AFB06B0BDE8F081000021
:1035B0003038024000080240000402400D4810B5B7
:1035C0000B4901600C49416000214FF48042816049
:1035D000C0E9031241618161C1610162FDF7EEFB47
:1035E000002803D0BDE81040FCF7A8BF10BD0000C4
:1035F0000054004020010020A0860100104810B5B2
:103600000E4901604FF48271416000210222816005
:10361000C0E90312012242615202C0E9062101629F
:10362000416281620A21C162FEF7A2FF002803D035
:10363000BDE81040FCF782BF10BD0000003800401C
:103640007401002010B592B000240F941C2108A82A
:103650001094FCF709FE20216846FCF705FE20487F
:103660001E4901606321C0E90114FA21C0E9031475
:1036700044618461FFF7DCF908B1FCF75FFF0F9448
:103680000FA917481094FFF705F908B1FCF756FF8A
:103690006020CDE908040A940B940C940D94082240
:1036A00008A90F480E94FFF75DF908B1FCF746FF33
:1036B00000944FF40050CDE9044002940194039427
:1036C000694607480794FFF7BAF808B1FCF736FFD8
:1036D0000348FFF71DF912B010BD000000000140C3
:1036E000CC01002010B500220F49104801F092F9DA
:1036F00008B1FCF723FF0E490C4801F0B5FB08B1F7
:10370000FCF71CFF0B49094800F00CFF08B1FCF75F
:1037100015FF064801F02CFC002803D0BDE810403E
:10372000FCF70CBF10BD000028000020340700206B
:10373000E80000207C000020334802F0CFFB334833
:1037400002F0CCFB324802F0C9FB324802F0C6FB63
:103750002F4802F0C3FB304802F0C0FB2A4802F0B9
:10376000BDFB2EA002F0BAFBFCF788FF2D4C002514
:1037700010B90120206000E025602BA002F0AEFB14
:1037800039A002F0ABFB48A002F0A8FB56A002F063
:10379000A5FB206810B164A002F0A0FB72A002F0AB
:1037A0009DFBFDF74BF8312806D0322807D033288F
:1037B00007D034280FD011E001F062FFDDE77AA0D6
:1037C00010E084A002F08AFB4FF47A70FDF7E0F875
:1037D00002F03CFED1E72068012806D020680028CE
:1037E0000FD087A002F07AFBC7E7FCF7FBFE0128A9
:1037F00003D00228C1D192A0F4E79CA002F06EFB96
:10380000BAE7A2A0EEE70000E0A00008FC9F0008D5
:10381000B09F000894A0000848A000080D0A0D0AF7
:10382000000000001C0000200D0A3D3D3D3D3D3DD7
:103830003D3D3D3D3D3D3D3D3D3D3D3D204D616975
:103840006E204D656E75203D3D3D3D3D3D3D3D3D10
:103850003D3D3D3D3D3D3D3D3D3D3D3D3D3D3D3D98
:103860003D3D3D0D0A0A00002020446F776E6C6FCD
:10387000616420496D61676520546F20746865201C
:1038800053544D33324634787820496E7465726EE5
:10389000616C20466C617368202D2D2D2D2D2D2DF2
:1038A00020310D0A0A000000202055706C6F616401
:1038B00020496D6167652046726F6D2074686520D0
:1038C00053544D33324634787820496E7465726EA5
:1038D000616C20466C617368202D2D2D2D2D2D2DB2
:1038E00020320D0A0A0000002020457865637574B7
:1038F0006520546865204E65772050726F6772614D
:103900006D202D2D2D2D2D2D2D2D2D2D2D2D2D2DB4
:103910002D2D2D2D2D2D2D2D2D2D2D2D2D2D2D2DD7
:1039200020330D0A0A000000202044697361626C94
:1039300065207468652077726974652070726F7491
:10394000656374696F6E202D2D2D2D2D2D2D2D2D40
:103950002D2D2D2D2D2D2D2D2D2D2D2D2D2D2D2D97
:1039600020340D0A0A0000003D3D3D3D3D3D3D3DFA
:103970003D3D3D3D3D3D3D3D3D3D3D3D3D3D3D3D77
:103980003D3D3D3D3D3D3D3D3D3D3D3D3D3D3D3D67
:103990003D3D3D3D3D3D3D3D3D3D3D3D3D3D3D3D57
:1039A0003D3D0D0A0A000000546869732066756E7B
:1039B0006374696F6E2069732064697361626C65FA
:1039C000642120506C656173652055736520310D4D
:1039D00000000000537461727420746F2065786574
:1039E00063757465207468652075736572206170F5
:1039F000706C69636174696F6E2E2E2E0D0A000063
:103A0000496E76616C6964204E756D626572202125
:103A1000203D3D3E20546865206E756D62657220C4
:103A200073686F756C64206265206569746865727F
:103A300020312C20322C2033206F7220340D0000D6
:103A40004572726F723A20466C61736820777269B2
:103A5000746520756E70726F74656374696F6E2023
:103A60006661696C65642E2E2E0D0A0057726974AA
:103A7000652050726F74656374696F6E206469733A
:103A800061626C65642E2E2E0D0A0000496E76610F
:103A90006C6964204E756D6265722021203D3D3E4B
:103AA00020546865206E756D6265722073686F754D
:103AB0006C642062652065697468657220312C2011
:103AC00032206F7220330D00FEE7FEE70148FDF75C
:103AD00011BE0000302600202DE9F04103680D469C
:103AE00004461E6C03EB4511D1F8080B94F806E070
:103AF0004FF400474FF0200C04F29C42BEF1010F3E
:103B000009D0DFF898E0764539D1020432D500BFFC
:103B1000C1F8087B3FE0224B5FEA007E04D59E425D
:103B200039D90004F4D436E05FEA806E02D5C1F8DA
:103B300008CB30E010F0280F2DD19E4201D90004AF
:103B4000E6D405EBC50004EB8000D1F8101BD0F8DB
:103B50007432C1F31201591AC0F8681200F51570D9
:103B6000ADB903691BB1C2681144C1600FE0012106
:103B700020680AE080060AD5C1F808CB07E035B90D
:103B8000D4F8640218B90021184601F035FFE9B2F3
:103B90002046FDF785FC0020BDE8F0810A31544F36
:103BA0000A30544F2DE9F84F0E4601EBC60100EBE9
:103BB000810481460568D4E909101434884202D989
:103BC0000120BDE8F88F081AA168814200D208469A
:103BD000C01C870805EB46181BE000BFA0EB010ADC
:103BE000A068504500D282460AF10300870899F880
:103BF000060000901FFA8AF3F2B22846E16802F04C
:103C0000A7FAE16801EB0A00E060616901EB0A00D4
:103C10006061D8F8180980B2B84205D3D4E904012C
:103C2000814201D20028D9D1D4E90401884208D8C0
:103C300006F00F0101208840D5F834188143C5F8FB
:103C400034180020BDE7704770B50C46054604E007
:103C5000284602F011F9012804D0641EF8D24FF072
:103C6000FF3070BD002070BD2DE9F84F884600215F
:103C70000646C8F80010924611466846FFF7E4FF72
:103C80004FF0FF39B0BB9DF80000182814D006DCB7
:103C9000012809D0022809D004282BD12EE0412880
:103CA00016D0612826D113E0802401E04FF480640F
:103CB00001253070671D15E051466846FFF7C4FFC7
:103CC000C0B99DF80000182814D1C8F8009015E07C
:103CD0000120BDE8F88F70195146FFF7B5FF48B9CC
:103CE0006D1CADB2BD42F6D3B178707881F0FF01A2
:103CF000884201D04846ECE7C8F800400020E8E7D9
:103D0000F8B515460E460B460092044601220221E4
:103D100000F02CF8A0B9134813490068B0FBF1F08B
:103D20004FF47A71484300906068B0F5827F0DD1FE
:103D30003346002280212046009500F017F870B12C
:103D4000606D40F0200060650320F8BD009830B140
:103D5000401E009020688068C0430006F6D5002011
:103D6000F8BD00001400002000366E012DE9F84374
:103D70001E46914688460446089DFDF719F8401BEB
:103D8000351AFDF715F8074625480068C0F3CB3013
:103D9000684338E0701C37D0FDF70AF8C01BA84212
:103DA00003D215B1009860B32CE02068416821F07F
:103DB000E00141606068B0F5827F0BD1A068B0F58A
:103DC000004F02D0B0F5806F04D12068016821F067
:103DD00040010160A06AB0F5005F09D12068016868
:103DE00021F4005101602068016841F40051016034
:103DF000012084F85100002084F850000320BDE821
:103E0000F8830025401E00902068816838EA010090
:103E100004D000214945BDD10020F0E70121F9E798
:103E20001400002070470178407841EA0020704774
:103E300070B5002204781346302C04D14478782CD5
:103E40000AD0582C08D06FF02F05845C74B36B2C0B
:103E50002ED04B2C2CD030E082780AB30224025DA5
:103E60005AB1A2F14105052D0AD9A2F16106052E2C
:103E700006D91135092D07D913E001200B6011E097
:103E8000A2F13006092E01D8303A04E0052D01D800
:103E9000373A00E0573A641C02EB03130B2CDED3D5
:103EA00002E000200B2C00D3002070BD0B6002E06C
:103EB0001AB1980207E0012015E06D2C01D04D2CBD
:103EC00003D112B118050860F5E7A4F13006092EF8
:103ED00008D803EB830305EB4303521C23440B2A4E
:103EE000B3D3E1E700200B2ADED270BDFDF7F8B9AD
:103EF00030B593B030216846FCF7B6F914210CA810
:103F0000FCF7B2F91C480025016841F080510160BE
:103F1000006800F0805011901848016841F4404159
:103F200001600068022400F44040119001200090DC
:103F3000000401908001CDE9064019200890C020BE
:103F4000CDE9090404200B906846FEF75BF908B13F
:103F500072B6FEE70CA90F2081E831004FF48050C3
:103F6000CDE90F0503210CA8FDF7D0FF002801D0F3
:103F700072B6FEE713B030BD40380240007000401A
:103F80000248016841F470010160704788ED00E06B
:103F9000F0B50268204B214C9F03214D214E9842E1
:103FA00007D0B84205D0A04203D0A84201D0B04209
:103FB00004D122F0700C4A6842EA0C02984210D0F8
:103FC000B8420ED0A0420CD0A8420AD0B04208D0CD
:103FD000154CA04205D0154CA04202D0144CA04272
:103FE00003D122F44074CA6822434C6922F0800253
:103FF000224302608A68C2620A688262984201D1E2
:1040000009690163012141610169C90703D001699F
:1040100021F001010161F0BD0000014000040040F9
:1040200000080040000C00400040014000440140F6
:104030000048014010B501F01F030121046A9940B6
:104040008C430462016A9A401143016210BD000072
:1040500030B5036A026A22F0010202624268846992
:1040600024F073050C682C4323F002058B682B4366
:104070000A4DA8420BD123F00805CB6822F4407208
:104080002B434D6923F0040315438A692A43426098
:10409000846149684163036230BD00000000014053
:1040A00030B5026A036A23F010030362436884692F
:1040B0000D6824F4E64444EA05248D6822F02002C9
:1040C00042EA05120B4DA8420ED1CD6822F08002C3
:1040D00042EA05124D6923F4406343EA85038D6982
:1040E00022F0400243EA85034360846149688163AA
:1040F000026230BD0000014030B5036A026A22F45A
:10410000807202624268C46923F4007324F073056C
:104110000C682C438D6843EA05230C4DA8420ED150
:10412000CD6823F4006343EA05234D6922F440522D
:1041300042EA05128D6923F4806342EA0512426067
:10414000C4614968C163036230BD000000000140E2
:1041500030B5046A026A22F4805202624268C3697E
:104160000D6823F4E64343EA05238D6824F40054E4
:1041700044EA0534064DA84204D14D6922F4804238
:1041800042EA85124260C36149680164046230BD3D
:10419000000001402DE9F0410C46D0F8D412D0F8CF
:1041A000C82200EB8101D1F8C01229B304F00F0638
:1041B00006EB860300EB83050027AB694BB106EBEA
:1041C000C60602EB8602D269B3FBF2F602FB163298
:1041D000A2B1C1F81472D0F8D42200EB8200D0F85A
:1041E000C40203692BB1D1F80802224601F504711B
:1041F00098470020BDE8F0810320FBE700231A4622
:104200002146AF6100F011FEF3E770B50546D0F826
:10421000D40205EB8000D0F8C04294B1284600F0EB
:10422000DAFCC4F80C02D5F8D412D4F8040205EB79
:104230008101D1F8C412CA6804F5037190470020C7
:1042400070BD032070BD000070B5224D0446297872
:1042500000F0FCFB2878002600F00F0000EB800047
:1042600004EB800086846978204600F0EFFB6878D4
:1042700000F00F0000EB800004EB8000A0F8646108
:10428000A978204600F0E2FBA87800F00F0000EBD0
:10429000800004EB80008684C684D4F8D40204EB4A
:1042A0008000D0F8C01299B1D0F8C40240688047AD
:1042B000D4F8D40204EB8000D0F8C00200F0E6FF8E
:1042C000D4F8D40204EB8000C0F8C062C4F8BC6229
:1042D000002070BD9400002010B5D0F8D41200EB7F
:1042E0008100D0F8C04284B1D0F8C41259B194F81A
:1042F0000002FF2807D08B6894F8012221469847D6
:10430000FF2084F80002002010BD032010BD000033
:104310000A210180004870479800002070B50646C9
:1043200082210C4800F015FB05460121094800F0E8
:1043300010FB04468121074800F00BFB0DB1102152
:10434000A971402104B1A18000B181804320308057
:10435000004870BDA400002070B5064682210D48BB
:1043600000F0F7FA054601210A4800F0F2FA044687
:104370008121084800F0EDFA0DB11021A9714FF428
:10438000007104B1A18000B18180432030800148D8
:1043900070BD0000A400002070B5064682210C48C4
:1043A00000F0D7FA05460121094800F0D2FA044688
:1043B0008121074800F0CDFA0DB11021A9714021EB
:1043C00004B1A18000B1818043203080004870BDDD
:1043D000A40000202DE9F04704464FF40775284655
:1043E00000F056FF06004FF0000863D02946FBF7A7
:1043F0003BFFD4F8D4023C4D04EB80004FF0100991
:10440000C0F8C062C4F8BC62207C4FF4007A012777
:10441000F0B3402302222978204600F048FC287897
:10442000402300F00F0000EB800004EB8000878445
:1044300002226978204600F03AFC6878082300F0F0
:104440000F0000EB800004EB80000322A0F86471F1
:10445000A978204601F00F0101EB810104EB8101F5
:10446000A1F82690A97800F022FCA87800F00F00AF
:1044700000EB800004EB80008784C6F80482D4F847
:10448000D402474604EB8000D0F8C402006800E084
:1044900018E006F5017680473761776132687AB1B6
:1044A000207CF8B140236978204600F00CFC002005
:1044B000BDE8F087D4F8D41204EB8101C1F8C082C2
:1044C0000220F5E7534602222978204600F0EFFB50
:1044D0002878534600F00F0000EB800004EB8000CA
:1044E0008784A5E75346DEE79400002010B5D0F896
:1044F000D41200EB8101D1F8C01259B1027C084CF2
:10450000002AD1F8042207D04023617800F0DBFBB9
:10451000002010BD032010BD4FF40073F5E700002C
:104520009400002039B1D0F8D42200EB8200C0F80A
:10453000C4120020704703207047D0F8D42200EB4B
:104540008200D0F8C00218B1C0F8041200207047F1
:1045500003207047D0F8D43200EB8300D0F8C002BB
:1045600028B1C0F81022C0F80812002070470320BC
:1045700070472DE9FC410646D0F8D4020C4606EB04
:1045800080000021D0F8C0728DF80010ADF8041042
:104590000D4637B1217811F060022FD0202A4BD17F
:1045A00002E00320BDE8FC81E288F2B109060DD5E6
:1045B000D0F8C40263783946D0F808C01846E047FE
:1045C000E288072A00D9072239462DE0607887F86B
:1045D0000002E088402800D34020C2B287F80122C0
:1045E0003946304600F081F82BE0D0F8C4026378F9
:1045F0000022866821461846B04722E0607830B134
:1046000001281ED00A2809D00B2815D110E096F8F1
:104610009C02032810D1022201A905E096F89C0211
:10462000032809D101226946304600F078F808E0F5
:1046300096F89C02032804D02146304600F04AF840
:1046400003252846AEE7000010B5D0F8D41200EBE1
:104650008101D1F8C02201211AB1D2F8143213B16C
:1046600016E0032010BD0121C2F814120949D2F846
:104670001032097801F00F0404EB840400EB840489
:10468000A361D2F81032D2F8082200F0CEFB00214C
:10469000084610BD9400002010B5D0F8B8220024C0
:1046A0005268904700B10324204610BD0020704797
:1046B00000207047134610B50A46002100F003FBA6
:1046C000002010BD134610B50A46002100F0ADFBD6
:1046D000002010BD10B50446802100F07EFB20466E
:1046E000BDE81040002100F078BB10B50323C0F8EE
:1046F0009432C0F858211346C0F85C210A460021C4
:1047000000F0E1FA002010BD10B50521C0F89412A8
:1047100000231A46194600F0D6FA002010BD10B545
:104720000223C0F8943282611346C2610A46002116
:1047300000F07BFB002010BD10B50421C0F89412DE
:1047400000231A46194600F070FB002010BD10B57A
:10475000044600F054FB012084F89C02D4F8B8020F
:1047600018B142682179204690470020C4F8C4025D
:10477000C4F8B402C4F8D0022046BDE8104000F0EE
:1047800010BA000010B50A46024903A000F00FF964
:10479000004810BD100A002043444320436F6E665A
:1047A0006967000012200880004870474800002018
:1047B00010B50A46024903A000F0F9F8004810BD00
:1047C000100A002043444320496E74657266616399
:1047D0006500000004200880004870474400002065
:1047E00010B50A46024903A000F0E1F8004810BDE8
:1047F000100A002053544D6963726F656C656374D1
:10480000726F6E696373000010B50A46024903A017
:1048100000F0CDF8004810BD100A002053544D336D
:1048200032205669727475616C20436F6D506F72DF
:104830007400000010B51A2008800A480168001DA5
:104840000468001D0068081809D008220649FEF710
:10485000C9FB0549042210312046FEF7C3FB02487C
:10486000801E10BD107AFF1F5E000020F8B50446C0
:104870000020ADF8000048880D46010A08295FD2E3
:10488000DFE801F05E0409175E5E3C45D4F8B4121F
:10489000207C0A6819E0207C02260028D4F8B8029F
:1048A00005D0C16A684688470146467039E0816A8A
:1048B000F8E7C0B2062843D2DFE800F0030A10147C
:1048C000181CD4F8B402426805E0694690471CE021
:1048D000D4F8B402826892B3207CF6E7D4F8B4022C
:1048E000C268F8E7D4F8B4020269F4E7D4F8B40275
:1048F0004269F0E7D4F8B4028269ECE7207CF0B9B1
:10490000D4F8B802416B68468847014609E0207C2C
:10491000A8B9D4F8B802016B684688470146072059
:104920004870EA888AB1BDF8000040B1824200D9DF
:104930000246ADF800202046FFF7F1FEF8BDFFE784
:1049400029462046FFF7C6FEF8E72046FFF7F4FEAB
:10495000F4E778B50E4642880178002504468A427D
:1049600012D9ADF800100AE0694600F019F8417854
:10497000052904D181780546B14205D0002561881A
:10498000BDF800209142EFD8284678BD01460020AE
:1049900002E0401CC0B2491C0A78002AF9D17047D5
:1049A0000A8803781A440A8001780844704770B571
:1049B00016460D46002820D00446FFF7E7FF0221E7
:1049C00001EB40014FF40070814204D82046FFF70C
:1049D000DDFF4000801C3080307828700320687034
:1049E0000220002206E02954401CC0B22A54401C78
:1049F000C0B2641C21780029F5D170BD01004FF0D0
:104A0000000004D0012901D0022901D00320704701
:104A10000120704778B10023C0F8B832C0F8C43222
:104A2000C0F8D03209B1C0F8B412012180F89C124C
:104A3000027000F0D5B80320704710B5D0F8C80256
:104A4000FCF783FDBDE81040FFF7D8BF10B5D0F8E4
:104A5000C802FCF755FDBDE81040FFF7CFBF2DE9B8
:104A6000F04117460446002521B194F89C02032822
:104A700042D04CE0D4F8941204F11400022935D14C
:104A8000D0E902639E4206D9F21A82603946204676
:104A9000FFF718FE0FE0B34214D14068984211D3DB
:104AA000D4F8981288420DD2002211462046FFF712
:104AB00009FEC4F8985200231A461946204600F011
:104AC00002F913E094F89C02032808D1D4F8B80244
:104AD000C16821B1C4F8D452C168204688478021FA
:104AE000204600F07AF92046FFF70EFE94F8A00267
:104AF00068B184F8A0520AE0D4F8B802426932B131
:104B0000C4F8D452426920469047002800D10020C2
:104B1000BDE8F08170B513460446002221B194F837
:104B20009C02032830D03AE0D4F8941204F5AA701D
:104B3000032934D1D0E902518D420AD96A1A826020
:104B40000846824200D3024619462046FFF7B2FDCE
:104B500025E094F8AA0210F01F0003D0012802D02B
:104B6000022800D0002294F89C02032808D1D4F82F
:104B7000B802016921B1C4F8D422016920468847EE
:104B80002046FFF7D9FD0AE0D4F8B802836933B1B3
:104B9000C4F8D422826920469047002800D1002022
:104BA00070BD10B5D0F8C802FCF784FCBDE8104019
:104BB000FFF724BF0020704710B50024012180F8C2
:104BC0009C12D0F8B82222B152680179904700B106
:104BD0000324204610BDD0F8C802FCF7E3BC000057
:104BE00010B5017839BB15490222C1F8E004C0F8BC
:104BF000C8124FF0A040086004200871CA7100205C
:104C000088714A728872C87208738873C8730846BC
:104C1000FDF726F808B1FBF791FC80210748FCF767
:104C20000CFC402200210548FCF70BFC80220121EE
:104C30000248FCF706FC002010BD000030260020D2
:104C40000A0601F07F01D0F8C80201EBC10100EBB8
:104C5000810001D5807D704790F85602704710B5ED
:104C6000D0F8D42200EB8202D2F8B82222B190F818
:104C70009C32032B02D004E0032010BD126A02B163
:104C80009047002010BD10B5D0F8D42200EB82026E
:104C9000D2F8B82222B190F89C32032B02D004E063
:104CA000032010BD526A02B19047002010BD10B51C
:104CB0001C461346D0F8C8022246FCF77CFCBDE82F
:104CC0001040FFF79BBE10B5D0F8C802FCF7A4FC5B
:104CD000BDE81040FFF792BE2DE9F0410026012506
:104CE000044680F89C52C4F894626660C4F8A462DA
:104CF00080F8A062D0F8B80230B1426822B1002139
:104D00002046904700B1032600224023114620464A
:104D1000FFF7CDFF4027A4F864513B4600228021D5
:104D20002046C4F86071FFF7C2FFA58430462762B1
:104D3000BDE8F08190F89C12042903D190F89D12EF
:104D400080F89C120020704710B590F89C1203293F
:104D500005D1D0F8B81211B1C96901B18847002056
:104D600010BD01740020704710B5D0F8C802FDF7DF
:104D700054F8BDE81040FFF741BE70B5044600F29C
:104D8000AA20054600F05AF80120C4F89402B4F8AD
:104D9000B002C4F8980294F8AA0210F01F010AD0D9
:104DA00001290ED0022912D000F080012046BDE872
:104DB000704000F012B829462046BDE8704000F06F
:104DC000D9B829462046BDE8704000F019BA2946F6
:104DD0002046BDE8704000F063B910B5D0F8C802B5
:104DE000FCF736FCBDE81040FFF708BE10B5D0F860
:104DF000C802FDF72CF8BDE81040FFF7FFBD10B565
:104E0000D0F8C802FDF744F8BDE81040FFF7F6BD42
:104E100090F89C12042903D090F89C1280F89D12FF
:104E2000042180F89C120020704710B5D0F8C80209
:104E3000FCF747FCBDE81040FFF7E0BD70B5054644
:104E400011F8010B2870087868704C1C2046FEF79A
:104E5000EAFF6880A41C2046FEF7E5FFA880A01C9E
:104E6000FEF7E1FFE88070BD38B504460020ADF8DC
:104E70000000A1B1C4F8B812D4F8D40204EB800049
:104E8000D0F8B802C16A19B168468847C4F8D002A0
:104E9000D4F8D802401CC4F8D802002038BD032042
:104EA00038BD02460020D2F8B832002B02D01B6871
:104EB00010461847704700002DE9F04188462B4EF8
:104EC0008978002504463170012906D941462046DB
:104ED000FFF700FC0320BDE8F08194F89C02022754
:104EE00002280CD003281DD041462046FFF7F2FBD4
:104EF00031782046FFF7D0FB03252846EBE789B33E
:104F000020466160FFF7CDFF050004D041462046F2
:104F1000FFF7E0FB1DE02046FFF70EFC032084F8BE
:104F20009C02EAE7C1B1606888421BD0C1B220464A
:104F3000FFF7B2FB317820466160FFF7B2FF050052
:104F400010D041462046FFF7C5FB21792046FFF7E8
:104F5000A3FB84F89C72D0E784F89C7220466160C1
:104F6000FFF79AFB2046FFF7E7FBC6E7900000201B
:104F7000FFF73CBF2DE9F0410A78002512F06002EE
:104F80000CD0202A01D0402A7DD1D0F8D42200EBC9
:104F90008202D2F8B8229268904731E04B78002222
:104FA00001260A2B6FD2DFE803F041666E586E08C7
:104FB000056E2D29FFF75AFC67E004468888D8B9AA
:104FC000C888C8B94888802816D200F07F0794F8AE
:104FD0009C02032810D084F89E7239462046FFF7C1
:104FE000C3FE2046FFF7A8FB1FB1022084F89C02F5
:104FF0004BE084F89C6248E0204644E0FFF75CFF09
:10500000054642E0CB88012B3DD190F89C32012B24
:1050100004D0022B02D0032B35D104E082600122A0
:1050200000F1080116E00122011D13E090F89C2216
:10503000012A03D0022A01D0032A24D1CA88022AD5
:1050400021D1C660D0F8A41209B10321C1600222A7
:1050500000F10C01FFF763FB17E04A88012A02D038
:10506000022A03D00FE0C0F8A46216E08988090A7A
:1050700080F8A01211E090F89C32012B08D0022B8E
:1050800006D0032B04D0FFF725FB2846BDE8F081AE
:1050900049880129F9D1C0F8A422FFF74DFBF4E7B4
:1050A0002DE9F041054608780C790E464FF00008CE
:1050B00010F060000BD0202801D040286AD1214692
:1050C0002846FFF7F3FAFF2800D0D8B395E07078B0
:1050D000C8B3012824D003285CD195F89C0202288B
:1050E00002D0032856D10CE0002C53D0802C51D094
:1050F00021462846FFF771FE80212846FFF76DFE06
:105100007BE0708840B93CB1802C05D0C88818B9C4
:1051100021462846FFF761FE2846FFF70DFB6CE0AD
:1051200095F89C020228DFD0032863D1708880BBE9
:10513000600603D021462846FFF77FFC2846FFF78C
:10514000FBFABCE700E00AE0C5F8D402D5F8B802E3
:105150008268F2B131462846904780464DE095F886
:105160009C020027022802D0032843D113E00CB18F
:10517000802C3FD1200604F07F0000EB800005EB7F
:10518000800101D5143101E001F5AA7102220F60FE
:105190002CE032E02EE0200604F00F0000EB80004F
:1051A00005EB800009D5808C20B304F07F0000EB74
:1051B000800005EB800614360AE0B0F86401C8B13F
:1051C00004F07F0000EB800005EB800606F5AA7670
:1051D0004CB1802C07D021462846FFF731FD10B195
:1051E0000120306000E03760022231462846FFF798
:1051F00096FA02E02846FFF76DFA4046BDE8F081D6
:1052000070B50546087800240E4610F0600003D003
:10521000202801D0402827D195F89C02012803D0EE
:10522000022801D003281FD1B088C1B201291AD8A1
:10523000C1B22846FFF73CFAFF280CD058B9D5F880
:10524000B8128A683AB1C5F8D4028A68314628464D
:105250009047044600E00324F088204307D1284605
:10526000FFF76AFA03E031462846FFF733FA204693
:1052700070BD10B50446FFF7C2FDD4F8B80218B1EE
:105280004268217920469047002010BD70470000F9
:10529000004870471024002070B50A78012302F0FE
:1052A0000F054E78AB401B4CD0F81C58012E17D080
:1052B00045EA0343C0F81C3800EB4210D0F8002B3D
:1052C00012040BD4D0F8002B0B890979C3F30A031D
:1052D0001A4344EA81410A43C0F8002B002070BD04
:1052E0009BB21D43C0F81C5800EB4210D0F80039A7
:1052F0001B04F3D4D0F800390D890979C5F30A05E8
:1053000089042B4341EA82510B432343C0F80039FF
:10531000E4E7000000800010D0F800196FF30A01E4
:10532000C0F80019D0F8041841F48071C0F80418CE
:105330000020704770B50D460446C2F3072104985B
:105340001E4601291BD0E06840F04000E060204686
:1053500000F032F8C6F307210029A16B26D021F412
:105360008031A163C5F30741012907D1A16841F04C
:105370000601A160A16841F02001A16070BDA16B90
:1053800021F48031A163E1680A4A1140E160E168DB
:1053900021F44011E160C0B2012803D1E06840F47B
:1053A0008010E060204600F007F8DBE741F4803130
:1053B000D7E70000BFFFBDFF08B500214FF07062C6
:1053C0000091009B5B1C009393420CD80369002B57
:1053D000F7DA0091016941F0010101610099491C6E
:1053E0000091914201D9032008BD0169C907F5D197
:1053F000002008BD30B54C780A78012300EB42123A
:10540000012C2CD0D2F8004B002C0BDAD2F8004B38
:1054100044F00064C2F8004BD2F8004B44F08044E2
:10542000C2F8004BD0F83C580C7804F00F0403FA93
:1054300004F425EA0444C0F83C48D0F81C48097834
:1054400001F00F018B4024EA0341C0F81C18D2F888
:10545000000B19490840C2F8000B002030BDD2F8FB
:105460000049002C0BDAD2F8004944F00064C2F87D
:105470000049D2F8004944F08044C2F80049D0F80D
:105480003C480D7805F00F0503FA05F5ADB2AC43C5
:10549000C0F83C48D0F81C48097801F00F018B4057
:1054A00099B28C43C0F81C48D2F80009034908405F
:1054B000C2F80009D1E700000078F3EF007833EC80
:1054C000D0F8001E21F00301C0F8001ED0F8041827
:1054D00021F00201C0F8041800207047D0F8001E27
:1054E00021F00301C0F8001ED0F8041841F00201B9
:1054F000C0F80418002070472DE9F04F00250E4633
:10550000044617462846294604EB8002C2F80411D7
:10551000401C0F28F8D3C3F307405FEA0009204678
:1055200016D0806B20F40012A263A06B40F400221E
:10553000A263084688462146C4F8000EC7F3072038
:10554000012817D00846D1F8001841F0030118E0EF
:10555000D0F8040840F00202C4F80428A06B40F41C
:105560000012A263A06B20F40022A263A06B20F4BF
:105570008022DDE7300E0846D1F8001801D041F056
:105580000101C0F80018102100F047FC00B101250E
:10559000204600F026FC00B101254046C4F81088E2
:1055A000C4F81488C4F81C8800214FF0006B4FF039
:1055B000904E4FF67F3AF2B215E000BF04EB411374
:1055C000D3F800C9BCF1000F06DA11B1C3F800E945
:1055D00004E0C4F800B901E0C3F80009C3F81009F9
:1055E000C3F808A9491C8A42E8D8002115E000BF89
:1055F00004EB4113D3F800CBBCF1000F06DA11B174
:10560000C3F800EB04E0C4F800BB01E0C3F8000BF2
:10561000C3F8100BC3F808AB491C8A42E8D8D4F889
:10562000101821F48072C4F81028A0616FF0804037
:105630006061C6F3074018B9A06940F01000A0618E
:10564000A0690A490843A061C7F3074018B1A069DF
:1056500040F00800A061B9F1010F03D1A06904492D
:105660000843A0612846BDE8F08F000000383C8068
:1056700004000040816821F0010181600020704732
:1056800070B542A292B007CA06AB83E8070042A0F9
:1056900000F024FC4FA000F021FC564D2846FAF7FC
:1056A000BDFF08B154A068E05EA000F017FC62A046
:1056B00000F014FC674800F0AFFD041E4EDD66A04C
:1056C00000F00CFC21462846FAF7AEFE05466D4870
:1056D000029003A94FF05A3081E8310002AE032056
:1056E000FAF7BAFF68480C90042231460CA8FAF782
:1056F000E5FF66A000F0F2FB6EA000F0EFFB78483B
:1057000000F0ECFB214606A8FDF74CFC75A000F06C
:10571000E5FB06A800F0E2FB75A000F0DFFB77A038
:1057200000F0DCFB09AC142277A10CA8FAF783FD8A
:1057300000200CA905F00F02C0F107038A5C2D09B7
:10574000401CE2540828F5DB0020207209A800F074
:10575000C5FB72A000F0C2FB76A00EE00320FAF7B2
:105760007BFF7BA000F0BAFB601C05D0A01C08D01A
:10577000E41C08D07BA000E082A000F0AFFB12B0D8
:1057800070BD90A0F9E796A0F7E700002020202048
:10579000202020202020000057616974696E672056
:1057A000666F72207468652066696C6520746F206E
:1057B00062652073656E74202E2E2E20287072650F
:1057C00073732027612720746F2061626F727429C0
:1057D0000A0D000045726173696E67204170706C3C
:1057E00069636174696F6E20417265612E2E2E0DA2
:1057F0000A000000000001084572726F723A2046EC
:1058000061696C656420746F2065726173652061E5
:1058100070706C69636174696F6E2061726561217B
:105820000D0A0000457261736520436F6D706C65F1
:1058300074652E0D0A0000005374617274696E67FE
:1058400020596D6F64656D20526563656976650AE0
:105850000D000000340200200A0A0D2046696C6524
:1058600020726563657074696F6E20636F6D706C14
:105870006574652E20566572696679696E672E2E8D
:105880002E0A0D00EFBEADDE00C00008566572693D
:105890006669636174696F6E20616E6420466C6135
:1058A0006720536574207375636365737366756CE5
:1058B000210D0A002D2D2D2D2D2D2D2D2D2D2D2D94
:1058C0002D2D2D2D2D2D2D2D2D2D2D2D2D2D2D2D08
:1058D0002D2D2D2D0D0A204E616D653A2000000002
:1058E000340600200A0D2053697A653A2000000032
:1058F0002042797465730D0A000000002043524372
:1059000033323A2030780000303132333435363794
:105910003839414243444546000000000D0A2D2D10
:105920002D2D2D2D2D2D2D2D2D2D2D2D2D2D2D2DA7
:105930002D0A0000506C65617365207265626F6F9F
:105940007420746865206465766963652E0D0A00AD
:105950000A0D55706772616465206661696C6564E3
:10596000210D0A000A0D4661696C656420746F2080
:1059700072656365697665207468652066696C6523
:10598000210A0D000A0A0D54686520696D6167657A
:105990002073697A65206973206869676865722079
:1059A0007468616E2074686520616C6C6F776564E3
:1059B000207370616365206D656D6F7279210A0DCA
:1059C000000000000A0A0D56657269666963617419
:1059D000696F6E206661696C6564210A0D000000C4
:1059E0000D0A0A41626F72746564206279207573D2
:1059F00065722E0A0D00000010B5036C134CA34213
:105A000003D9D0F8003B002B1EDB0023C0F8103B6D
:105A1000D0F8103B43F40023C0F8103BD0F8103B03
:105A200043F01803C0F8103BD0F8103B43F0C043DC
:105A3000C0F8103B012907D1C0F8142BD0F8001B87
:105A400041F08021C0F8001B002010BD0A30544FE7
:105A50004A780B78012A00EB43100BD0D0F8002BCA
:105A600022F40012C0F8002B0979032914D002296E
:105A700012D017E0D0F8002922F40012C0F8002953
:105A80000979032901D002290CD1D0F8001941F07D
:105A90008051C0F8001905E0D0F8001B41F080519A
:105AA000C0F8001B002070470A784B78D1B200EB99
:105AB0004110012B12D0D0F8001B002906DB2AB1BF
:105AC000D0F8001B21F08041C0F8001BD0F8001B6B
:105AD00041F40011C0F8001B00207047D0F80019F5
:105AE000002906DB2AB1D0F8001921F08041C0F866
:105AF0000019D0F8001941F40011C0F80019EBE7C3
:105B0000F8B50C784F788B4DE3B26FF0604600EB40
:105B10004313012F29D0D3F8107B6FF31207C3F87A
:105B2000107BD3F8107B2F40C3F8107B002C7DD066
:105B30000D69002D7BD08C6825446D1EB5FBF4F5F6
:105B4000ADB26C430C62D3F8104B06EAC5452C434A
:105B5000C3F8104BD3F8104B0D6AC5F312052C4354
:105B6000C3F8104B012A70D0CBE00F69EFB1D3F826
:105B700010796FF31207C3F81079D3F810792F401A
:105B8000C3F810790CB30F698D682F447F1EB7FBE3
:105B9000F5F5D3F81079ADB206EAC5463743C3F838
:105BA00010790E79012E1CD02AE0D3F810692E400E
:105BB000C3F81069D3F8105945F40025C3F81059FB
:105BC000D3F810596FF3120520E00E698D68AE42CC
:105BD00000D90D61D0F8105945F40026C0F81069BD
:105BE0000EE0D3F8106926F0C046C3F81069D3F868
:105BF00010694FF0C04707EA45752E43C3F8106996
:105C0000D3F810590E69C6F312063543C3F810597C
:105C1000012A1BD000EB4413D3F8004944F004449C
:105C2000C3F800490C79012C31D001E044E057E081
:105C30000A695AB3D0F83428097801F00F0301211A
:105C400099400A43C0F8342871E056E0CA691AB195
:105C500000EB4413C3F81429097901290ED1D0F8B7
:105C60000818C90500EB4411D1F8002902D442F00C
:105C7000005201E042F08052C1F8002900EB4410CC
:105C8000D0F8001941F00441C0F800194FE0D0F8F5
:105C90000848E405D3F8004902D444F0005401E078
:105CA00044F08054C3F8004900920A8A93B20A78FB
:105CB000C96800F04DFA3AE00C690CB18C680C61CF
:105CC0008C680C62D0F8105BC4F312042543C0F852
:105CD000105BD0F8104B44F40024C0F8104B41E79F
:105CE000D3F8104B8D68C5F312052C43C3F8104B45
:105CF000D3F8104B44F4002432E7CA680AB1C3F861
:105D0000142B097901290CD1D0F80808C005D3F863
:105D1000000B02D440F0005001E040F08050C3F886
:105D2000000BD3F8000B40F00440C3F8000B002038
:105D3000F8BD0000FFFF07E038B5002200921346CF
:105D40004D780A7842F2107400EB4212012D19D0FE
:105D5000D2F8005B002D3CDAD2F8005B45F000651C
:105D6000C2F8005B0A7800EB4212D2F8005B45F003
:105D70008045C2F8005B009A521C0092A24221D9D1
:105D8000012326E0D2F80059002D22DAD2F800597A
:105D900045F00065C2F800590A7800EB4212D2F8CB
:105DA000005945F08045C2F80059009A521C0092F3
:105DB000A242E5D80A7800EB4212D2F80029002A64
:105DC000F3DB06E00A7800EB4212D2F8002B002A3F
:105DD000D1DB184638BD816841F0010181600020A7
:105DE000704708B500214FF070620091009B5B1C6A
:105DF000009393420AD80369002BF7DA009110212F
:105E000001610099491C0091914201D9032008BD0C
:105E10000169C906F5D4002008BD18B500224FF06D
:105E200070630092009C641C00949C420CD804692E
:105E3000002CF7DA0092202242EA811101610099D8
:105E4000491C0091994201D9032018BD01698906B6
:105E5000F5D4002018BDD0F8080810F0060004D0D2
:105E6000022803D0062801D00F2070470220704777
:105E7000406900F00100704709490A8809490B8808
:105E80009A420AD0084A0B88D25C02700888401CEB
:105E9000C0F30A000880012070470020704700000E
:105EA0007600002078000020100C0020094991F8AD
:105EB0009C22032A0CD1D1F8BC1200BFD1F81422C5
:105EC000002AFBD10449087001210348FAF796BA69
:105ED00070470000340700201800002070B50B4DFB
:105EE000064695F89C0203280ED13046FAF7C7F90A
:105EF000044603E095F89C02032805D1A1B2304680
:105F0000FAF77CFA0128F5D070BD000034070020B4
:105F1000D0F81818D0F81C08084080B27047D0F8A4
:105F20001818D0F81C080840000C704710B5D0F8BD
:105F30001038D0F8342801F00F0400EB4110E24093
:105F400002F00102D0F8080943EAC212104010BD65
:105F500000EB4111D1F8081BD0F814080840704735
:105F6000416980690840704730B503460846940887
:105F700002F00301002203F5805303E01D6840F89E
:105F8000045B521CA242F9D300290BD01C680022EA
:105F9000D50024FA05F3491E521C090400F8013B00
:105FA000090CF5D130BD70B50446C068002520F05D
:105FB000C040E060012901D079B120E0E06840F004
:105FC0000050E0600A20FAF7E3FC60690A3510F03F
:105FD000010F10D1C82DF5D30DE0E06840F08040EE
:105FE000E0600A20FAF7D4FC60690A3510F0010F6E
:105FF00001D0C82DF5D3C82D01D0002070BD0120DF
:1060000070BDD0F8002822F4FE62C0F80028D0F855
:1060100000284FF4FE6303EA01110A43C0F8002888
:1060200000207047022A3ED1264A274B0A449A4252
:1060300001D20F2138E0254A254B0A449A4201D269
:106040000E2131E0234A244B0A449A4201D20D2109
:106050002AE0224A224B0A449A4201D20C2123E030
:10606000204A214B0A449A4201D20B211CE01F4ACC
:106070001F4B0A449A4201D20A2115E01D4A1E4BC9
:106080000A449A420FD31D4A1D4B0A449A4201D238
:10609000082109E01B4A11441B4A914201D2072101
:1060A00002E0062100E00921C26822F47052C260B9
:1060B000C2684FF4705303EA81210A43C260002092
:1060C00070470000405327FF00350C00401E1BFFA7
:1060D00040420F0000DC0BFF804F1200808CF9FE65
:1060E00020D6130060B6E5FE60E3160000D3CEFEB6
:1060F00040771B00C05BB3FEC091210000CA91FE37
:1061000020753800E05459FEE09C410010B504466B
:1061100000214FF67F3000BF04EB4112C2F808099E
:10612000C2F8080B491C0F29F6D30020C4F8100848
:10613000C4F81408C4F81C082046FFF752FE0028D3
:1061400005D12046BDE810401021FFF766BE10BD06
:1061500010B5029C74B9DB1C9C0800EB02300023D4
:1061600000F5805004E000BF51F8042B02605B1C76
:10617000A342F9D3002010BD30B587B01421684682
:10618000FAF772F80E480021026842F0010202603C
:1061900000684FF4805400F0010000940590012045
:1061A000CDE90101074D039169462846FAF706FD3E
:1061B000002221462846FAF7F6FD07B030BD000060
:1061C000303802400000024010B51048FFF751F887
:1061D0000E48FEF7BCFA0E4C206840F080002060AC
:1061E0000A20FAF7D5FB206820F0800020600848DC
:1061F0002030016821F0800101600448D0F8C80215
:10620000FBF794FDBDE81040FFF7B6BF3407002050
:1062100014380240FEE700002DE9F04FADF22C4D9E
:106220004FF0000ADFF864B10446CDF808A45546E3
:10623000D0464FF480174FF0FF39CDF810B4CDF8A9
:1062400014A400263A460DF20C416846FDF70CFDF9
:1062500098B1012875D0B8F1000F00DD6D1C052D37
:1062600071DD1820FFF722FE5FF01800FFF71EFE19
:1062700000200DF22C4DBDE8F08FDDF80C24002538
:106280004A4507D042B19DF80100F1B288420BD0D7
:10629000152078E00620E9E70620FFF707FEDDF885
:1062A00014040028CDD05AE0BEB120460DF1030100
:1062B000F9F7C1FFDDF80C042146C0F38D020DF59E
:1062C0008260FAF7FBF9D8B31820FFF7EFFD18202A
:1062D000FFF7ECFD6FF00100CBE79DF8030088B3FA
:1062E00000212B4A0DF1030002E05354401C491CCD
:1062F00003780BB1FF29F8DD02F801A000210DF5AC
:106300008362401C02E05354401C491C0378202B3C
:1063100001D01029F7DB02F801A00DF581611046CC
:10632000FDF786FDDDF808046FF4E021C8420BD9C3
:106330001820FFF7BBFD1820FFF7B8FD484698E787
:1063400010E016E008E01DE05846FAF767F906206D
:10635000FFF7ACFD432006E00620FFF7A7FDDDF8C0
:10636000080486E70620FFF7A1FD4FF00108761C20
:1063700068E71820FFF79AFD1820FFF797FD6FF0E8
:10638000020076E74320FFF791FD5BE7000001087C
:10639000340600200907090E002804DB00F1E02084
:1063A00080F80014704700F00F0000F1E02080F842
:1063B000141D704702E008C8121F08C1002AFAD154
:1063C00070477047002001E001C1121F002AFBD175
:1063D0007047000010B50420FCF711FA06484FF48E
:1063E0007A710078B1FBF0F004490968BDE810400B
:1063F000B1FBF0F0FCF70FBA0800002014000020F9
:1064000070B5054600244FF47A7603E0304600F07C
:1064100004F8641CAC42F9D370BD70B54FF0E023B2
:1064200000215C6900EB40009A694501986990423F
:10643000FCD002D2A2EB000202E0A4EB0006324440
:1064400011440246A942F1D370BD000010B5FFF718
:10645000BBFE4FF4FA70FAF79BFAFBF7F1FDFAF77F
:1064600073FA4FF0E021002008614861886172B63C
:1064700005494868054A90605060096881F30888BA
:10648000BDE8104000470000000001081C0000208B
:106490000EB54B494FF000600860FAF729FFFDF791
:1064A00027FDFDF737F8FDF7A9F8FDF7CBF8FDF765
:1064B00085F8FDF717F9FDF71BF8FFF78BFFFCF7E1
:1064C000ADFD08213F48FCF7F5FAFCF751FE00242A
:1064D000F0231A46214620460094FCF7E7FD0A20E7
:1064E000FFF78EFF3220FCF71DFF0025F9F7B9FFFB
:1064F00058B9F9F7EBFF0546F9F7E8FF28B132A0E4
:10650000FFF7ECFC0020F9F7FBFFDFF8DC9001213E
:106510004846FAF743FC18264FF6FF784FF4FA770F
:1065200000B175B13846FFF76BFF01214846FAF715
:1065300035FC08B1002D3FD0CDE90046434602941A
:1065400027E02A4B04CB93E82300294B9A4202D13F
:10655000B0F15A3F26D027A0FFF7C0FCCDE9004696
:10656000454643462EA250214A200294FCF772FF72
:10657000CDE900462B462CA2802118200294FCF77E
:1065800069FF4FF4FA60FAF703FACDE900462B46AB
:1065900002942AA250214820FCF75CFFFAF784F805
:1065A000F9F7D0FE2848F9F73FFF854204D127A02C
:1065B000FFF794FCFFF74AFF3846FAF7E9F9FBE7E3
:1065C00008ED00E0CC010020656E746572206669FC
:1065D000726D7761726520757064617465206D6F8E
:1065E00064650D0A000000000000024000C00008C1
:1065F000EFBEADDE4E6F2041707020666F756E6429
:106600002C20656E746572206669726D77617265A3
:1066100020757064617465206D6F64650D0A0000FB
:106620004E6F204170702100506C7A20446F776E5D
:106630006C6F61642041505000000000426F6F7425
:106640006C6F6164000000000000010856616C6915
:10665000642041505020666F756E642C206A756D01
:1066600070696E6720746F206170706C696361740B
:10667000696F6E2E2E2E0D0A000000000000000033
:1066800000000000000000000000040404040400F6
:106690000004000014140A000000000000000000C4
:1066A00000000A0A1F0A0A1F0A0A000000040E1549
:1066B00005060C14150E0400000012150D152E2CE5
:1066C0002A1200000000040A0A36151529160000D7
:1066D0000202010000000000000000001008080491
:1066E0000404040408081000020404080808080848
:1066F0000404020000000004150E0E150400000042
:1067000000000008083E080800000000000000002B
:10671000000000000202010000000000003F000035
:106720000000000000000000000000000002000067
:1067300000201010080804040202010000000E11DD
:1067400011111111110E00000000040604040404CC
:10675000040E000000000E1111080402011F0000C9
:1067600000000E11100C1010110E00000000080C9B
:106770000C0A091F081C000000001F01010F111066
:10678000110E000000000C12010D1311110E00007B
:1067900000001E10080804040404000000000E118C
:1067A000110E1111110E000000000E11111916101A
:1067B00009060000000000000400000000040000C2
:1067C00000000000000400000004040000001008A5
:1067D0000402020408100000000000003F003F0017
:1067E000000000000000020408101008040200006D
:1067F00000000E11110804040004000000001C2217
:10680000292D2D1D221C0000000004040C0A0A1E64
:106810001233000000000F12120E1212120F0000AD
:1068200000001E1101010101110E000000000F12F5
:1068300012121212120F000000001F120A0E0A029A
:10684000121F000000001F120A0E0A0202070000B9
:1068500000001C1201013911120C0000000033125B
:10686000121E12121233000000001F04040404045C
:10687000041F000000003E0808080808080809076F
:10688000000037120A060A12123700000000070241
:1068900002020202223F000000003B1B1B1B1515D9
:1068A0001535000000003B1216161A1A12170000C8
:1068B00000000E1111111111110E000000000F1235
:1068C000120E02020207000000000E111111111732
:1068D000190E180000000F12120E0A1212370000D3
:1068E00000001E1101060810110F000000001F1506
:1068F00004040404040E00000000331212121212E9
:10690000120C000000003312120A0A0C04040000EA
:106910000000151515150E0A0A0A000000001B0AD2
:106920000A04040A0A1B000000001B0A0A0A0404E5
:10693000040E000000001F0908040402121F0000DA
:106940001C0404040404040404041C0000020204E3
:1069500004040808081010000E08080808080808B1
:1069600008080E00040A00000000000000000000FB
:1069700000000000000000000000003F02040000D2
:10698000000000000000000000000000000C121CCD
:10699000123C000000030202020E1212120E00004E
:1069A00000000000001C1202120C00000018101061
:1069B000101C1212123C000000000000000C121EFD
:1069C000021C000000182404041E0404041E00001D
:1069D00000000000003C120C021C221C00030202FA
:1069E000020E121212370000000404000006040414
:1069F000040E000000080800000C0808080808073A
:106A000000030202021A0A060A1300000007040427
:106A100004040404041F000000000000000F15150A
:106A20001515000000000000000F121212370000C0
:106A300000000000000C1212120C00000000000008
:106A4000000F1212120E020700000000001C1212AA
:106A5000121C103800000000001B06020207000094
:106A600000000000001E020C101E000000000004C8
:106A7000041E0404041C000000000000001B12128D
:106A8000123C000000000000001B0A0A0404000081
:106A9000000000000015150E0A0A000000000000AA
:106AA000001B0A040A1B0000000000000033121241
:106AB0000C08040300000000001E0804041E00006F
:106AC00018080808080C080808081800080808082A
:106AD0000808080808080808060404040408040450
:106AE0000404060016090000000000000000000079
:106AF0000000000000000000000000000000000096
:106B0000000000080808080808080000181800001D
:106B100000486C241200000000000000000000008B
:106B20000000002424247F1212127F12121200008F
:106B30000000081C2A2A0A0C1828282A2A1C0808DF
:106B400000000022251515152A585454542200001F
:106B50000000000C1212120A76252911916E000015
:106B60000006060403000000000000000000000012
:106B700000402010100808080808081010204000E5
:106B80000002040808101010101010080804020079
:106B90000000000008086B1C1C6B080800000000C7
:106BA00000000000080808087F0808080800000026
:106BB00000000000000000000000000006060403C2
:106BC0000000000000000000FE00000000000000C7
:106BD00000000000000000000000000006060000A9
:106BE0000000804040202010100808040402020029
:106BF000000000182442424242424242241800004F
:106C0000000000080E08080808080808083E0000F0
:106C10000000003C4242422020100804427E000056
:106C20000000003C4242201820404042221C00004C
:106C3000000000203028242422227E20207800001A
:106C40000000007E0202021A26404042221C000080
:106C5000000000382402021A264242422418000092
:106C60000000007E22221010080808080808000012
:106C70000000003C4242422418244242423C0000B0
:106C8000000000182442424264584040241C000086
:106C90000000000000001818000000001818000094
:106CA00000000000000000080000000000080804C8
:106CB00000000040201008040204081020400000DA
:106CC0000000000000007F0000007F0000000000C6
:106CD00000000002040810204020100804020000F8
:106CE0000000003C424246402010100018180000EE
:106CF0000000001C225A555555552D42221C0000FB
:106D00000000000808181414243C224242E7000046
:106D10000000001F2222221E22424242221F0000A7
:106D20000000007C4242010101010142221C0000DE
:106D30000000001F2242424242424242221F000003
:106D40000000003F4212121E12120242423F000097
:106D50000000003F4212121E12120202020700003F
:106D60000000003C2222010101712122221C0000AE
:106D7000000000E7424242427E42424242E70000B7
:106D80000000003E0808080808080808083E00003F
:106D90000000007C10101010101010101010110FB7
:106DA0000000007722120A0E0A1212222277000037
:106DB000000000070202020202020202427F0000FB
:106DC00000000077363636362A2A2A2A2A6B000037
:106DD000000000E346464A4A5252526262470000AF
:106DE0000000001C2241414141414141221C000060
:106DF0000000003F424242423E02020202070000FF
:106E00000000001C2241414141414D53321C6000B1
:106E10000000003F4242423E1212222242C70000BE
:106E20000000007C4242020418204042423E000022
:106E30000000007F4908080808080808081C00002E
:106E4000000000E74242424242424242423C0000CD
:106E5000000000E74242222424141418080800000D
:106E60000000006B4949494955553622222200004D
:106E7000000000E7422424181818242442E70000E8
:106E8000000000772222141408080808081C0000DB
:106E90000000007E2120101008040442423F000040
:106EA0000078080808080808080808080808780092
:106EB00000000202040408080810102020204040AE
:106EC000001E1010101010101010101010101E00C6
:106ED0000038440000000000000000000000000036
:106EE000000000000000000000000000000000FFA3
:106EF0000006080000000000000000000000000084
:106F0000000000000000003C4278444242FC0000C7
:106F1000000000030202021A26424242261A000022
:106F20000000000000000038440202024438000063
:106F300000000060404040784442424264D8000073
:106F4000000000000000003C427E0202423C0000C3
:106F5000000000F08808087E08080808083E0000C5
:106F6000000000000000007C22221C023C42423C47
:106F7000000000030202023A4642424242E7000099
:106F80000000000C0C00000E08080808083E000075
:106F90000000003030000038202020202020221E59
:106FA0000000000302020272120A16122277000089
:106FB0000000000E0808080808080808083E00003D
:106FC000000000000000007F9292929292B70000B1
:106FD000000000000000003B4642424242E7000041
:106FE000000000000000003C42424242423C0000DF
:106FF000000000000000001B26424242221E020741
:10700000000000000000007844424242447840E022
:1070100000000000000000774C040404041F00007E
:10702000000000000000007C42023C40423E0000A4
:10703000000000000008083E0808080808300000AA
:1070400000000000000000634242424262DC000097
:1070500000000000000000E742242414080800009B
:1070600000000000000000EB4949555522220000B5
:10707000000000000000007624181818246E00009C
:1070800000000000000000E742242414180808074C
:10709000000000000000007E22100808447E00006E
:1070A00000C0202020202010202020202020C000F0
:1070B00010101010101010101010101010101010D0
:1070C000000608080808081008080808080806004C
:1070D0000C32C200000000000000000000000000B0
:1070E00000000000000000000000000000000000A0
:1070F0000000000000000000000000000000000090
:10710000000000000000000000000000000000007F
:1071100000000000000000006000600060006000EF
:10712000600060006000400020002000200000009F
:10713000000000006000600060000000000000002F
:1071400000000000600660063003980188004400DB
:10715000000000000000000000000000000000002F
:10716000000000000000000000000000000000001F
:1071700000000000000000001002100210021002C7
:10718000FE07FE0708020801080108010801FE07C2
:10719000FE070401040104010401000000000000D6
:1071A00000000000000040004000F00158034C03C4
:1071B000CC034C0058007000E000C001C001400347
:1071C0004C035C034C034801F00040004000000009
:1071D00000000000000000000E010A019100910073
:1071E0009100510051003A00AE03A0025004500437
:1071F000480448044804840284030000000000009E
:10720000000000000000000038006C006C006C0002
:107210006C006C002C0098071C011A01330133012B
:107220006301E300C308C6093C070000000000003A
:10723000000000000C001C001000100008000400FA
:10724000000000000000000000000000000000003E
:10725000000000000000000000000000000000002E
:1072600000000000000400020001800080004000D7
:1072700040002000200020002000200020002000EE
:107280004000400080008000000100020004000077
:1072900000000000020004000800100010002000A0
:1072A00020004000400040004000400040004000FE
:1072B0002000200010001000080004000200000060
:1072C0000000000000000000000000004000C000BE
:1072D0004000460C4E0FD001F0015E0F460C4000FE
:1072E000400040000000000000000000000000001E
:1072F000000000000000000000000000000040004E
:107300004000400040004000FE0F400040004000B0
:1073100040004000000000000000000000000000ED
:10732000000000000000000000000000000000005D
:10733000000000000000000000000000000000004D
:10734000000000000C001C001000100008000400E9
:10735000000000000000000000000000000000002D
:107360000000000000000000FE0700000000000018
:10737000000000000000000000000000000000000D
:1073800000000000000000000000000000000000FD
:1073900000000000000000000000000000000000ED
:1073A000000000001C001C001C0000000000000089
:1073B00000000000000400060002000300010001BC
:1073C000800080004000400060002000200010008D
:1073D0001000080008000C00040006000200000075
:1073E00000000000000000000000F00098010C0305
:1073F0000C0306060606060606060606060606062A
:1074000006060C030C039801F000000000000000C9
:107410000000000000000000000040007C00600050
:10742000600060006000600060006000600060005C
:107430006000600060006000FC03000000000000CD
:1074400000000000000000000000F80084010203BA
:1074500006030603000300018001C0006000200055
:107460001000080204020602FE03000000000000F3
:10747000000000000000000000007800C600860147
:10748000860180018001C0007000800100010003BE
:107490000003060306038601F80000000000000058
:1074A0000000000000000000000080018001C00119
:1074B000A001A00190018801880184018201FE0FD2
:1074C0008001800180018001E007000000000000D1
:1074D00000000000000000000000FC0304000400A5
:1074E000040004000400F4008C0104030003000302
:1074F0000603060382018401F8000000000000007A
:1075000000000000000000000000E00118030C0370
:107510000C0004000600E60116030E060606060629
:10752000060604060C021803F0000000000000002C
:1075300000000000000000000000F8070C06040234
:107540000401000100018000800040004000400074
:10755000600060006000600060000000000000004B
:1075600000000000000000000000F8010C03060607
:10757000060606060C021C03F000C8010C030606F2
:107580000606060606060C03F001000000000000D7
:1075900000000000000000000000F0000C010C03DF
:1075A000060206060606060606078C06780600068C
:1075B000000300030C018C017800000000000000B3
:1075C00000000000000000000000000000000000BB
:1075D00000000000E000E000E0000000000000000B
:1075E00000000000E000E000E000000000000000FB
:1075F000000000000000000000000000000000008B
:1076000000000000600060000000000000000000BA
:10761000000000000000600060004000200020002A
:1076200000000000000000000004000200018000D3
:107630004000200010000800040008001000200096
:107640004000800000010002000400000000000073
:10765000000000000000000000000000000000002A
:1076600000000000FE07000000000000FE07000010
:10767000000000000000000000000000000000000A
:1076800000000000000000000400080010002000BE
:1076900040008000000100020004000200018000A0
:1076A000400020001000080004000000000000005E
:1076B00000000000000000000000E0031806040CB9
:1076C000040C0C0C0C0C0007800140004000400032
:1076D00000000000E000E000E0000000000000000A
:1076E0000000000000000000E00018030C02CC05C0
:1076F00064056605A605B604B604B604B604B6026B
:10770000E4010C040C021803F0000000000000006B
:107710000000000000000000000060006000500059
:10772000D00090009000880088010801F80104034F
:1077300004030402020202060F0F00000000000012
:1077400000000000000000000000FE008C030C039D
:107750000C030C030C038C01FC000C030C020C0644
:107760000C060C060C060C03FE01000000000000D5
:1077700000000000000000000000E00318030C06F9
:107780000C040404060006000600060006000600BD
:1077900006040C040C021803F000000000000000B6
:1077A000000000000000000000007F008C010C03BE
:1077B0000C030C060C060C060C060C060C060C063C
:1077C0000C060C030C038C017F000000000000007D
:1077D00000000000000000000000FF030603060494
:1077E0000604060086008600FE00860086008600ED
:1077F0000600060406040602FF0300000000000065
:1078000000000000000000000000FF030603060463
:107810000604060086008600FE00860086008600BC
:1078200006000600060006001F0000000000000021
:1078300000000000000000000000F00018010C0231
:107840000C0204020600060006000600C60F06032E
:1078500006030C030C031803F000000000000000F6
:10786000000000000000000000000F0F06060606E2
:107870000606060606060606FE07060606060606AF
:1078800006060606060606060F0F000000000000AA
:1078900000000000000000000000FC036000600029
:1078A00060006000600060006000600060006000D8
:1078B0006000600060006000FC0300000000000049
:1078C00000000000000000000000F807C000C00039
:1078D000C000C000C000C000C000C000C000C000A8
:1078E000C000C000C000C000C000C60066003C0070
:1078F00000000000000000000000CF038601C60069
:1079000046002600160036002E006E004600C60017
:1079100086008601060106038F07000000000000B4
:10792000000000000000000000001F00060006002C
:107930000600060006000600060006000600060017
:107940000600060406040602FF0300000000000013
:107950000000000000000000000007078603860307
:107960008E038E034E034E034A035A035A033A030F
:1079700032033203320312038707000000000000C5
:10798000000000000000000000008E0F0C021C022E
:107990001C0234023402640264024402C4028402FF
:1079A00084038403040304031F020000000000009A
:1079B00000000000000000000000F00098010C032F
:1079C0000C02060606060606060606060606060655
:1079D00006060C020C039801F000000000000000F5
:1079E00000000000000000000000FF000603060683
:1079F00006060606060606068603FE0006000600C4
:107A000006000600060006001F000000000000003F
:107A100000000000000000000000F00098010C03CE
:107A20000C020606060606060606060606060606F4
:107A300076064C02CC039801F0008007000300009A
:107A400000000000000000000000FF010603060621
:107A50000606060606060603FE004600C600860069
:107A600086010603060306060F0E00000000000054
:107A700000000000000000000000F8020C030602F5
:107A8000060206000E003C00F800E0038003000739
:107A90000206020606060C03F001000000000000CA
:107AA00000000000000000000000FE076204610802
:107AB00061086000600060006000600060006000BD
:107AC0006000600060006000F8010000000000003D
:107AD000000000000000000000001E070C020C0265
:107AE0000C020C020C020C020C020C020C020C0226
:107AF0000C020C020C021801F00000000000000053
:107B0000000000000000000000000F070602040152
:107B100004010C010C0188008800980098005000B6
:107B20005000700030002000200000000000000025
:107B300000000000000000000000F70E6204420494
:107B40004604460464026402E402E4029C029C01CE
:107B5000980198018801880088000000000000005A
:107B6000000000000000000000009E070C0108015A
:107B700018019000B0006000200060006000D0009C
:107B800090008801080104038E0700000000000037
:107B9000000000000000000000000F0F06040402B7
:107BA0000C0208011801B800B0007000600060000D
:107BB0006000600060006000F8010000000000004C
:107BC00000000000000000000000FC070C0206039B
:107BD00002018001800040004000200020001000D1
:107BE000180008040C040402FE030000000000005A
:107BF00000000000E0032000200020002000200002
:107C00002000200020002000200020002000200074
:107C1000200020002000200020002000E0030000C1
:107C2000000000000000000004000400080008003C
:107C30001000100010002000200040004000C00094
:107C40008000800000010001000200020002000428
:107C5000000000007C004000400040004000400068
:107C60004000400040004000400040004000400014
:107C70004000400040004000400040007C00000008
:107C800000006000900008010000000000000000FB
:107C900000000000000000000000000000000000E4
:107CA00000000000000000000000000000000000D4
:107CB00000000000000000000000000000000000C4
:107CC00000000000000000000000000000000000B4
:107CD0000000000000000000000000000000FF0F96
:107CE000000000001800600000000000000000001C
:107CF0000000000000000000000000000000000084
:107D00000000000000000000000000000000000073
:107D10000000000000000000000000000000000063
:107D200000000000F0010C030C030003E0031C033F
:107D30000E03060306038E0B7C0E000000000000FD
:107D4000000000000000000008000E000C000C0005
:107D50000C000C00CC013C031C060C060C060C06A7
:107D60000C060C060C021C03E401000000000000DD
:107D70000000000000000000000000000000000003
:107D800000000000F0008C018C0186010600060056
:107D9000060006020C020C01F000000000000000CA
:107DA00000000000000000000002C0030003000308
:107DB0000003000378038C030C0306030603060389
:107DC0000603060304038C0778010000000000008E
:107DD00000000000000000000000000000000000A3
:107DE00000000000E001180308020C060C06FC0766
:107DF0000C000C0018041802E00100000000000054
:107E000000000000000000000000C0036006300613
:107E100030003000FE013000300030003000300013
:107E20003000300030003000FC0100000000000095
:107E30000000000000000000000000000000000042
:107E400000000000F007D8068C018C018C0198011D
:107E5000F8000C00FC00CC03060306038E03F800B8
:107E6000000000000000000008000E000C000C00E4
:107E70000C000C00EC011C030C030C030C030C03A2
:107E80000C030C030C030C039E0700000000000011
:107E90000000000000000000000060006000000022
:107EA000000040007C006000600060006000600036
:107EB0006000600060006000FC0300000000000043
:107EC00000000000000000000000C001C001000030
:107ED00000000001F001800180018001800180012B
:107EE000800180018001800180018001CC007C0044
:107EF000000000000000000008000E000C000C0054
:107F00000C000C008C038C008C004C006C005C009E
:107F10008C008C010C010C039E0700000000000087
:107F2000000000000000000040007C0060006000D5
:107F30006000600060006000600060006000600041
:107F40006000600060006000FC03000000000000B2
:107F50000000000000000000000000000000000021
:107F6000000000003707EE0666066606660666062F
:107F70006606660666066606FF0F00000000000043
:107F800000000000000000000000000000000000F1
:107F900000000000EE011C030C030C030C030C0397
:107FA0000C030C030C030C039E07000000000000F0
:107FB00000000000000000000000000000000000C1
:107FC00000000000F00098010C03060606060606F5
:107FD000060606060C030C03F0000000000000007B
:107FE0000000000000000000000000000000000091
:107FF00000000000EE011C030C060C060C060C062B
:108000000C060C060C031C03EC010C000C003E00DB
:108010000000000000000000000000000000000060
:108020000000000078028C030C030603060306031D
:108030000603060304038C03780300030003C00750
:108040000000000000000000000000000000000030
:10805000000000009F03580638061800180018009A
:108060001800180018001800FF00000000000000B1
:108070000000000000000000000000000000000000
:1080800000000000F0031C030C020C023800F0009A
:10809000C003040304038C03FC0100000000000083
:1080A0000000000000000000000000002000200090
:1080B00030003000FE013000300030003000300071
:1080C0003000300030023002E0010000000000000B
:1080D00000000000000000000000000000000000A0
:1080E000000008028E030C030C030C030C030C03AA
:1080F0000C030C030C039C07780100000000000037
:10810000000000000000000000000000000000006F
:10811000000000001E070C02080108011801900071
:10812000B000B0006000600020000000000000000F
:10813000000000000000000000000000000000003F
:1081400000000000F70E6204460464026402EC02C0
:108150009C019801980198010800000000000000AF
:10816000000000000000000000000000000000000F
:1081700000000000BC0718011001B00060006000A2
:10818000E0009000080108039E07000000000000C6
:1081900000000000000000000000000000000000DF
:1081A000000000009E0708010801080190009000EF
:1081B000B0006000600060002000200024001C006F
:1081C00000000000000000000000000000000000AF
:1081D00000000000FC018401C40044006000200095
:1081E0003000180208020C03FC010000000000002F
:1081F00000000000000380008000800080008000FC
:10820000800080008000400020004000800080004E
:10821000800080008000800080008000000300005B
:10822000400040004000400040004000400040004E
:10823000400040004000400040004000400040003E
:10824000400040004000400040004000400040002E
:10825000000000000C0010001000100010001000C2
:10826000100010001000200040002000100010003E
:108270001000100010001000100010000C00000092
:1082800000001C002204C204800300000000000063
:1082900000000000000000000000000000000000DE
:1082A00000000000000000000000000000000000CE
:1082B00000000000000000000000000000000000BE
:1082C00000000000000000000000000000000000AE
:1082D000000000000000000000000000000000009E
:1082E000000000000000000000000000000000008E
:1082F00000000000000000000000C001C001C0013B
:10830000C001C001C001C001800080008000800069
:10831000800080008000000000000000000080015C
:10832000C003C00380010000000000000000000046
:10833000000000000000E01CE01CF01E700E38077A
:108340001803080184000000000000000000000085
:10835000000000000000000000000000000000001D
:10836000000000000000000000000000000000000D
:10837000000000000000000000000000201020109D
:10838000201020102010FE7FFE7F1008100810081B
:108390001008100810081008FE7FFE7F080408046B
:1083A00008040804080400000000000000000000A9
:1083B000000000000000000000010001C00760197B
:1083C000103118311839183938017001E001C00333
:1083D0008007000F001D003900311C311C310C31A9
:1083E0000C11180DE0070001000100010000000061
:1083F0000000000000000000000000001C10361803
:108400006308630C63046304630263026301361D43
:108410009C37802280634063406320632063306325
:1084200010221836081C00000000000000000000A8
:10843000000000000000000000000000F0009801B3
:108440008C018C018C018C018C00CC007800183ED2
:108450001C083608320863046304C304C30383435F
:1084600006438E26781C000000000000000000007B
:108470000000000000001C003C003C003000300008
:1084800010000C00060000000000000000000000CA
:1084900000000000000000000000000000000000DC
:1084A00000000000000000000000000000000000CC
:1084B0000000000000000040002000100008000C38
:1084C0000004000600030003000380018001800116
:1084D000800180018001800180010003000300030E
:1084E00000060006000C00080010002000400000FC
:1084F000000000000000020004000800100030002E
:1085000020006000C000C000C00080018001800128
:1085100080018001800180018001C000C000C00096
:10852000600060003000100008000400020000003D
:10853000000000000000000000000000000000003B
:1085400000018003800300011C713C79783DC00765
:108550000001C007783D3C791C7100018003800355
:10856000800100000000000000000000000000008A
:1085700000000000000000000000000000000000FB
:1085800000000001000100010001000100010001E4
:10859000FC7F000100010001000100010001000159
:1085A00000000000000000000000000000000000CB
:1085B00000000000000000000000000000000000BB
:1085C00000000000000000000000000000000000AB
:1085D000000000000000000000000000000000009B
:1085E0001C003C003C003000300010000C00060075
:1085F000000000000000000000000000000000007B
:10860000000000000000000000000000000000006A
:10861000FE7F0000000000000000000000000000DD
:10862000000000000000000000000000000000004A
:10863000000000000000000000000000000000003A
:10864000000000000000000000000000000000002A
:108650000000000000000000000000000000180002
:108660003C003C001800000000000000000000007A
:1086700000000000000000400060002000300010FA
:1086800000180008000C00040006000200030001AE
:1086900080018000C0004000600020003000100019
:1086A000180008000C000400060002000000000092
:1086B000000000000000000000000000C007600C87
:1086C00030181830183018200C600C600C600C60EA
:1086D0000C600C600C600C600C60182018301830B6
:1086E0003018600CC007000000000000000000000F
:1086F00000000000000000000000000000018001F8
:10870000F8018001800180018001800180018001E9
:108710008001800180018001800180018001800151
:108720008001C003F81F00000000000000000000EE
:10873000000000000000000000000000E007101C26
:108740000818043004300C300C30003000180008D9
:1087500000040002000180004000202010200820BA
:108760000430FC1FFC1F000000000000000000009F
:10877000000000000000000000000000E003180EF0
:108780000C0C0C180C180C180018000C0006C00378
:10879000000E00180010003000300C300C300C10AF
:1087A0000C18180CE003000000000000000000009E
:1087B000000000000000000000000000000C000E9F
:1087C000000E000F800E800E400E600E200E100E68
:1087D000100E080E040E040EFE7F000E000E000E9A
:1087E000000E000E000EC07F000000000000000020
:1087F000000000000000000000000000F03FF03F1B
:1088000010001000100008000800C807280C1818F5
:10881000081000300030003000300C300C300418EC
:108820000418080CF0030000000000000000000025
:10883000000000000000000000000000800FC010D9
:10884000203010301800180008000C008C0F6C1835
:108850003C301C600C600C600C600C6018601820D0
:1088600030306018C0070000000000000000000069
:10887000000000000000000000000000F83FF83F8A
:108880001C100C080408040400040002000200018B
:1088900000010001800080008000C000C000C00016
:1088A000C000C000C0000000000000000000000088
:1088B000000000000000000000000000E007300C95
:1088C00018180C300C300C301C3038187008E007C9
:1088D000B007180E0C1C063806300630063006307D
:1088E0000C18180CE003000000000000000000005D
:1088F000000000000000000000000000E003180479
:108900000C080C1806100630063006300630063803
:108910000C3C1836F03100300018001800180C0C10
:108920000C060C03F0010000000000000000000035
:108930000000000000000000000000000000000037
:10894000000000000000000000008001C003C00320
:108950008001000000000000000000000000800115
:10896000C003C00380010000000000000000000000
:1089700000000000000000000000000000000000F7
:1089800000000000000000000000C000C000000067
:1089900000000000000000000000000000000000D7
:1089A0000000C000C00080008000400040000000C7
:1089B000000000000000000000000020001000087F
:1089C0000004000600038001C000600030001800B1
:1089D0000C00180030006000C00080010003000699
:1089E000000400080010002000000000000000004B
:1089F0000000000000000000000000000000000077
:108A000000000000000000000000FE7F00000000E9
:108A1000000000000000FE7F0000000000000000D9
:108A20000000000000000000000000000000000046
:108A3000000000000000000000000400080010001A
:108A400020006000C000800100030006000C001838
:108A500000300018000C000600038001C000600018
:108A600020001000080004000000000000000000CA
:108A700000000000000000000000C00730180830AF
:108A800008600C601C601C601C600030001C00064C
:108A90000001800080008000800000000000800154
:108AA000C003C003800100000000000000000000BF
:108AB000000000000000000000000000C007601877
:108AC000103018200C2F8C4D864CC64CC64C664C72
:108AD00066446644662666266615CC1C0C40082053
:108AE00018303018C007000000000000000000002F
:108AF000000000000000000000000001C001C001F3
:108B0000C00140016003200320032003300610064B
:108B100010061006F80F080C080C080C0C0C0418B2
:108B2000041806181F7C0000000000000000000070
:108B3000000000000000000000000000FE07181CFC
:108B4000183818301830183018301818180CF80762
:108B5000181818301820186018601860186018600D
:108B600018301818FE0F0000000000000000000080
:108B7000000000000000000000000000C027603876
:108B8000103018200C400C400400060006000600BF
:108B9000060006000600060006000C400C400C20F3
:108BA00018303018C007000000000000000000006E
:108BB000000000000000000000000000FE03180E8E
:108BC00018181830183018301860186018601860BD
:108BD0001860186018601860186018301830181085
:108BE0001818180EFE03000000000000000000002E
:108BF000000000000000000000000000FE3F1830F0
:108C0000182018601840180018081808180CF80FD9
:108C1000180C1808180818001800180018401840F8
:108C200018201830FE3F0000000000000000000087
:108C3000000000000000000000000000FE7F18702F
:108C4000184018C018801800181018101818F81FAD
:108C5000181818101810180018001800180018001C
:108C6000180018007E000000000000000000000056
:108C7000000000000000000000000000C013701C95
:108C8000101018100C200C2004000600060006002E
:108C90000600060006FC063006300C300C3018309A
:108CA00018303008C007000000000000000000007D
:108CB0000000000000000000000000003F7E0C18D3
:108CC0000C180C180C180C180C180C180C180C1884
:108CD000FC1F0C180C180C180C180C180C180C187D
:108CE0000C180C183F7E000000000000000000007F
:108CF000000000000000000000000000F81F8001DC
:108D0000800180018001800180018001800180015B
:108D1000800180018001800180018001800180014B
:108D200080018001F81F000000000000000000002A
:108D3000000000000000000000000000E07F0006CE
:108D400000060006000600060006000600060006F3
:108D500000060006000600060006000600060006E3
:108D600000060006000600060E060E038E01FC003B
:108D70000000000000000000000000007E7C1818C9
:108D80001808180418061802180198019801D8014B
:108D9000B803380318071806180E180C181C1818F2
:108DA000183018307EFC00000000000000000000B9
:108DB0000000000000000000000000007E0018001D
:108DC00018001800180018001800180018001800E3
:108DD0001800180018001800180018001840184053
:108DE00018201830FE3F00000000000000000000C6
:108DF0000000000000000000000000001FF81C3808
:108E00001C381C381C3C343434343434343674321A
:108E10006432643264326431C431C431C431C43028
:108E2000C43084309FFC00000000000000000000FF
:108E30000000000000000000000000001F7C1C106B
:108E40003C103410341074106410E410C410C411B9
:108E500084118413041304170416041E041C041C38
:108E6000041C04181F18000000000000000000008F
:108E7000000000000000000000000000C003300CF3
:108E8000181808100C300C3006600660066006608A
:108E9000066006600660066006600C200C30081054
:108EA0001818300CC0030000000000000000000093
:108EB000000000000000000000000000FE0F181875
:108EC000183018601860186018601860183018188A
:108ED000F80F1800180018001800180018001800E3
:108EE000180018007E0000000000000000000000D4
:108EF000000000000000000000000000C003300C73
:108F000018180C100C300C20066006600660066015
:108F100006600660066006600660E4612C331C3261
:108F20001816300EC007004C007C0038000000000E
:108F3000000000000000000000000000FE07181CF8
:108F4000183818301830183018301818180CF8075E
:108F500098031803180718061806180E180C180C92
:108F6000181C18187E7800000000000000000000A7
:108F7000000000000000000000000000E027303882
:108F800018300C200C200C000C0018007800E003B6
:108F9000800F001E003800700060046004600860EC
:108FA00018303818C80F0000000000000000000052
:108FB000000000000000000000000000FC3F8C21C9
:108FC00084618241824180018001800180018001B1
:108FD0008001800180018001800180018001800189
:108FE00080018001E0070000000000000000000098
:108FF0000000000000000000000000003F7C0C109A
:109000000C100C100C100C100C100C100C100C1080
:109010000C100C100C100C100C100C100C100C1070
:1090200008083804E0030000000000000000000011
:109030000000000000000000000000003EF81820C2
:1090400018201820301030103010301060086008E0
:109050006008E00CC004C004C004800380038003E7
:10906000800300010001000000000000000000007B
:10907000000000000000000000000000DFF3866137
:10908000862186218C210C218C238C138C138C132C
:109090004C1358125816580E380E380E380E300C25
:1090A0001004100410040000000000000000000084
:1090B0000000000000000000000000007E3E1808D4
:1090C00038083004300470026002E001C001C001C1
:1090D000800180034003400720062006100C100C7E
:1090E000081808183E7C0000000000000000000086
:1090F0000000000000000000000000007E7C1C104A
:10910000181018083008300C700460046002C002A7
:10911000C002C001800180018001800180018001C6
:1091200080018001E0070000000000000000000056
:10913000000000000000000000000000F83F1818C8
:109140000818040C040E00060007000380038001C9
:10915000C001C000E000600070003000382018201E
:109160001C100C18FE1F0000000000000000000092
:10917000000000000000C03F4000400040004000F0
:1091800040004000400040004000400040004000DF
:1091900040004000400040004000400040004000CF
:1091A00040004000400040004000C03F0000000080
:1091B0000000000000000000000008001800180077
:1091C000100030002000600060004000C0008000FF
:1091D0008001800100010003000200060006000477
:1091E000000C0008001800180010003000200000DB
:1091F000000000000000FC03000200020002000268
:10920000000200020002000200020002000200024E
:10921000000200020002000200020002000200023E
:1092200000020002000200020002FC030000000035
:109230000000000000008007C00620081010000099
:10924000000000000000000000000000000000001E
:10925000000000000000000000000000000000000E
:1092600000000000000000000000000000000000FE
:1092700000000000000000000000000000000000EE
:1092800000000000000000000000000000000000DE
:1092900000000000000000000000000000000000CE
:1092A0000000000000000000000000000000FFFFC0
:1092B0000000000000007800C00000010000000075
:1092C000000000000000000000000000000000009E
:1092D000000000000000000000000000000000008E
:1092E000000000000000000000000000000000007E
:1092F000000000000000000000000000000000006E
:1093000000000000000000000000F00318060C0C34
:109310000C0C000C800F700C1C0C0C0C060C060CBA
:10932000064C0C4FF8380000000000000000000060
:109330000000000000000000000010001E001800E7
:1093400018001800180018001800180FD818383026
:10935000386018601860186018601860186018206D
:1093600038307818C8070000000000000000000036
:1093700000000000000000000000000000000000ED
:1093800000000000000000000000C007700C18186A
:1093900018180C180C000C000C000C000C201820E5
:1093A00018103008C0070000000000000000000096
:1093B000000000000000000000000010001E001867
:1093C00000180018001800180018E01B301C1818AE
:1093D00018180C180C180C180C180C180C18081865
:1093E000181C307AE00900000000000000000000B6
:1093F000000000000000000000000000000000006D
:1094000000000000000000000000C007300C181829
:1094100008100C300C30FC3F0C000C000C00182025
:1094200018107018C00700000000000000000000C5
:10943000000000000000000000000000003E80C3AB
:1094400080C0C0C0C000C000C000FC1FC000C00081
:10945000C000C000C000C000C000C000C000C0000C
:10946000C000C000F80F0000000000000000000075
:1094700000000000000000000000000000000000EC
:1094800000000000000000000000C077306C1018E1
:109490001818181818181018300CF00718001800B1
:1094A000F00FF03F08700C600C600C603838E00F73
:1094B0000000000000000000000010001E00180066
:1094C00018001800180018001800980FD818383025
:1094D000183018301830183018301830183018304C
:1094E000183018307EFC0000000000000000000072
:1094F0000000000000000000000000008003800366
:1095000080030000000000000001F80180018001DC
:109510008001800180018001800180018001800143
:1095200080018001F81F0000000000000000000022
:1095300000000000000000000000000000380038BB
:1095400000380000000000000010801F0018001804
:10955000001800180018001800180018001800184B
:1095600000180018001800180018180C1806F0034E
:109570000000000000000000000010001E001800A5
:1095800018001800180018001800183E180C1806CB
:10959000180318019801D801380318071806180C89
:1095A000181C18187E7C000000000000000000005D
:1095B000000000000000000000000001F801800130
:1095C0008001800180018001800180018001800193
:1095D0008001800180018001800180018001800183
:1095E00080018001F81F0000000000000000000062
:1095F000000000000000000000000000000000006B
:1096000000000000000000000800EE1C9C338C31BC
:109610008C318C318C318C318C318C318C318C3162
:109620008C318C31DE7B0000000000000000000067
:10963000000000000000000000000000000000002A
:10964000000000000000000010001E0FD818383085
:1096500018301830183018301830183018301830CA
:10966000183018307EFC00000000000000000000F0
:1096700000000000000000000000000000000000EA
:1096800000000000000000000000C007701C103047
:1096900018300C600C600C600C600C600C601830B2
:1096A00018303018C0070000000000000000000063
:1096B00000000000000000000000000000000000AA
:1096C000000000000000000010009E0F5818383005
:1096D000182018601860186018601860186018303A
:1096E00038307818980718001800180018007E0005
:1096F000000000000000000000000000000000006A
:1097000000000000000000000000C023303C1838BA
:1097100018300C300C300C300C300C300C30083061
:109720001838303CE033003000300030003000FCAE
:109730000000000000000000000000000000000029
:10974000000000000000000060007E3C6066606178
:10975000E000E00060006000600060006000600009
:1097600060006000FE070000000000000000000034
:1097700000000000000000000000000000000000E9
:1097800000000000000000000000E0273038183022
:10979000182018007000E003800F001C0430043013
:1097A0000C301C18EC0F000000000000000000004E
:1097B00000000000000000000000000000000000A9
:1097C000800080008000C000E000FC1FC000C000DE
:1097D000C000C000C000C000C000C000C000C02069
:1097E000C0208011000F00000000000000000000F9
:1097F0000000000000000000000000000000000069
:10980000000000000000000010201E3C183018303E
:109810001830183018301830183018301830183008
:10982000183830F4E01300000000000000000000D1
:109830000000000000000000000000000000000028
:10984000000000000000000000007E3C181818080E
:10985000380830043004700260026002E001C00188
:10986000C001C000800000000000000000000000F7
:1098700000000000000000000000000000000000E8
:1098800000000000000000000000DFF78E630C23E2
:109890008C238C239813981358165816700E700E3C
:1098A000700E2004200400000000000000000000F2
:1098B00000000000000000000000000000000000A8
:1098C00000000000000000000000FC3E7008700472
:1098D000E004C002C0018003800340076006200C42
:1098E000100C18183E7E0000000000000000000070
:1098F0000000000000000000000000000000000068
:10990000000000000000000000007E7C181818080D
:1099100030083008300460046004C002C002C00295
:109920008001800180018000800080004C003C00AC
:109930000000000000000000000000000000000027
:1099400000000000000000000000FC1F0C0C040ED2
:109950000406000380038001C000E0007020302076
:1099600038301C18FC1F0000000000000000000040
:1099700000000000000000300008000400040004A3
:1099800000040004000400040004000400040002B9
:10999000800100020004000400040004000400042C
:1099A000000400040004000400040008003000006B
:1099B000000100010001000100010001000100019F
:1099C000000100010001000100010001000100018F
:1099D000000100010001000100010001000100017F
:1099E000000100010001000100010001000100016F
:1099F0000000000000000C001000200020002000EB
:109A00002000200020002000200020002000400036
:109A100080014000200020002000200020002000C5
:109A20002000200020002000200010000C0000007A
:109A300000003800C400864002610022001C0000C3
:109A40000000000000000000000000000000000016
:109A50000000000000000000000000000000000006
:109A600000000000000000000000000000000000F6
:109A7000D6D0200020002000FE0322022202220273
:109A8000FE032202200020002000BEB0FC010401E1
:109A9000FC010401FC012000FF070401FC0120007F
:109AA00024013202D4B0FE070204FA0402040204C4
:109AB000FE05520452044A0586050204FE07B5E776
:109AC00010001000FF0111011101FF01110111012E
:109AD000FF0111041004E007D7D30000FC0180004F
:109AE000400020002000FF07200020002000200070
:109AF0003800D6D08000800080008000FC1F8410D9
:109B00008410841084108410FC1F84108000800056
:109B100080008000BEB0F80F0808F80F0808F80FA2
:109B20008000FF7F0000F80F08080808F80F800089
:109B30008410A2204000D4B00000FE3F0220F22793
:109B400002200220FA2F2221222122211229122969
:109B50000A2E0220FE3F0220B5E780008000800030
:109B6000FC1F841084108410FC1F84108410841047
:109B7000FC1F845080408040007FD7D30000FE1F30
:109B800000080004000280018000FF7F8000800048
:109B90008000800080008000A0004000D6D000003F
:109BA0000000000000180000080000080000080085
:109BB000080818F8FF1F18081818081818081818A7
:109BC0000818180818180818F8FF1F0808080008CF
:109BD000000008000008000008000018000018003D
:109BE000001800000000BEB00000000000004000AF
:109BF00006C0FF07400006C0FF07400006C0FF0781
:109C0000400802003000FEFF3F000000C0FF07C018
:109C10000002C00002C00002C0FF038010008011DB
:109C20000160100E3010180C1E30001C00000000E7
:109C3000D4B0000000000000080030F8FF1F08004A
:109C40001008C010083F100800100800100800138A
:109C5000C8FF10082210082210082210082210083D
:109C6000211208211488601648C01328001008002B
:109C700010F8FF1F080010000000B5E7000000000A
:109C80000000001800000800000800000800F0FFB5
:109C90000F100804100804100804100804F0FF074F
:109CA000100804100804100804100804F0FF07103E
:109CB000080000081000081000082000183000F00C
:109CC0001F000000D7D3000000000000000004F0D7
:109CD000FF0F00000600000100C00000280000186F
:109CE00000001800001830FEFF7F00180000180068
:109CF00000180000180000180000180000180000EC
:109D00001800001800001F00000C00000000D6D052
:109D10000000000000000000008000000080010042
:109D2000008001000080010000800100008001002F
:109D30001080010CF0FFFF0F30800104308001041F
:109D4000308001043080010430800104308001043F
:109D50003080010430800104F0FFFF0730800104EF
:109D600030800104008001000080010000800100BB
:109D700000800100008001000080010000800100DF
:109D80000080010000800100008000000000000051
:109D9000BEB0000000000000000000000000000154
:109DA000800100FFFF01000380010003800100FF2C
:109DB000FF01000380010003800100FFFF0100811B
:109DC0008100000003000000031CFCFFFF3F0000B7
:109DD00040000003C00100FFFF010003C0000003BA
:109DE000C0000003C00000FFFF00000141000004AC
:109DF0000100000E71000007810180010107600071
:109E0000010E1898011C04E0011800C000000000B9
:109E10000000D4B0000000000000000000000008B6
:109E2000F0FFFF1F3000000C3000000C3000100C61
:109E300030FE3F0C3004000C3000000C3000000CF1
:109E40003000000C3000C00CF0FFFF0D3030060E6B
:109E50003030060C3010060C3010060C3010060C9A
:109E60003018860C3018860C3008060D300C860D24
:109E70003006EE0F3002FC0D3001000CF000000C3B
:109E80003000000CF0FFFF0F3000000C1000000449
:109E900000000000B5E7000000000000000000C066
:109EA000000000C0010000C0000000C0000000C0B1
:109EB000000000C00000E0FFFF0360C0000360C0BE
:109EC000000360C0000360C0000360C0000360C006
:109ED0000003E0FFFF0360C0000360C0000360C038
:109EE000000360C0000360C00003E0FFFF0360C028
:109EF000000160C0000000C0000800C0001000C0E9
:109F0000001000C0001800C001380080FF1F0000D2
:109F1000000000000000D7D3000000000000000097
:109F20000000000000000003C0FFFF0700008007E2
:109F30000000C000000060000000180000000C00DD
:109F40000080030000800300008001000080010801
:109F50000080011CFCFFFF3F008001000080010029
:109F600000800100008001000080010000800100ED
:109F700000800100008001000080010000800100DD
:109F8000008001000080010000FC010000E00000F2
:109F90000040000000000000000000000000000081
:109FA000010203040607080900000000010203047F
:109FB0000D0A3D20202020202020202020202020AD
:109FC0002020202020202020202020202020202091
:109FD0002020202020202020202020202020202081
:109FE0002020202020202020202020202020202071
:109FF000202020202020203D000000000D0A3D20D0
:10A00000202020202020202020202020202843291C
:10A0100020434F5059524947485420323031312063
:10A0200053544D6963726F656C656374726F6E69CA
:10A03000637320202020202020202020202020208A
:10A040002020203D000000000D0A3D20202020207F
:10A050002020202020202020202020202020202000
:10A060002020202020202020202020202020427975
:10A07000204D4344204170706C69636174696F6E58
:10A08000205465616D202020202020202020203DAC
:10A09000000000000D0A3D202053544D3332463459
:10A0A000787820496E2D4170706C69636174696FB6
:10A0B0006E2050726F6772616D6D696E67204170BE
:10A0C000706C69636174696F6E20202856657273C5
:10A0D000696F6E20312E302E3029203D00000000A7
:10A0E0000D0A3D3D3D3D3D3D3D3D3D3D3D3D3D3D03
:10A0F0003D3D3D3D3D3D3D3D3D3D3D3D3D3D3D3D90
:10A100003D3D3D3D3D3D3D3D3D3D3D3D3D3D3D3D7F
:10A110003D3D3D3D3D3D3D3D3D3D3D3D3D3D3D3D6F
:10A120003D3D3D3D3D3D3D3D000000004CA1000852
:10A130000000002020010000B46300086CA20008A9
:10A1400020010020F8390000C4630008000000006E
:10A1500000000000010000001000000000000000EE
:10A160000024F400000000000000000000000000D7
:10A1700000000000A5470008D5470008E147000897
:10A18000094800083548000885470008B14700081D
:10A190000403090412010002020200408304405734
:10A1A00000020102030100001A0300000000000089
:10A1B000000000000000000000000000000000009F
:10A1C0000000000000000000950300088F03000855
:10A1D0008B030008B9030008F90300080000000021
:10A1E000810182000A060002000000400100000018
:10A1F00009024300020100C032090400000102020A
:10A2000001000524001001052401000104240202BC
:10A210000524060001070582030800100904010057
:10A22000020A000000070501024000000705810244
:10A2300040000000D543000849420008734500086B
:10A2400000000000D9420008954100080B420008B8
:10A25000000000000000000000000000594300085A
:0CA260001D43000899430008114300084A
:040000050800019955
:00000001FF
